:020000041100E9
:10300000002373B52B4D2C4C28006361022601F080
:1030100071F94021FE2221742800284B009601F00E
:10302000BBF9002836D1217CFF222800244B0096D2
:1030300001F0B2F900282DD1224BA2899A4226D163
:10304000E389214A93420DD1204B6361204B2268D2
:10305000002A03D1002B01D043CB43C4280001F048
:1030600087F973BD1B4A934201D00023EFE71A4B47
:103070001A4A1B68934206D9C02304222800217CE7
:103080009B0001F0FFF9114B6361154BDFE7002353
:103090002374EAE7CC233821AC2228009B01217459
:1030A00001F0F0F90028F2D10E4B63610E4BE38181
:1030B0000E4BCCE7D441FF1FA861FF1FB461FF1F77
:1030C000B661FF1F5959000083050000214100111E
:1030D00058BD001182150000CC61FF1F871300004E
:1030E00064BD0011D9410011AAAAFFFF4CBD001117
:1030F000F7B5164B0192C318021D002000938823D8
:103100005B05D3181B685C1C1AD09CB2402C18D8E5
:103110008D781E0CAC466746CD782D023D43AE42FD
:1031200006D1019800280ED110000C70240A4C70B2
:1031300003249BB20733A343D218009B9A42DED3E9
:10314000FEBD4432F9E71000FAE7C046FC0F00006C
:10315000802213B503000324019189B25201073183
:103160009B18A14304305A1A88235B05C3181B68B7
:10317000591C03D190429241104016BD99B240298A
:1031800007D80B000733A343C0189042ECD30020AC
:10319000F3E74430F9E7134B134A1B68126810B584
:1031A000FA24934201D81A00F824104BE4021B6859
:1031B0009A4210D813000E4A12689A420ED3013375
:1031C00007D1F823DB029C4203D10A49054808F0E5
:1031D00057FB200010BDFC24E402ECE7FE24E402CF
:1031E000F7E7C04600C0071100D0071100E0071143
:1031F00000F00711FFFFFF7FF0B59BB015000490B2
:103200000391402A00D9A0E006AB59801A80FFF74D
:10321000C2FF0400042816D9002206A9FFF768FFA0
:10322000052810D906AB1B88AB420CD1002D07D066
:10323000514B2A000499C01808F0F2FA002802D174
:1032400001201BB0F0BD06AB1D8020000699FFF7E2
:103250007FFF041E7BD1069B0793FFF79CFF802313
:103260005B01C618802307001B039E4201D3F8268A
:10327000F60288235B05F31801931B68013302D023
:10328000019808F03DFB3D49019808F0F9FA3B1D13
:103290000293331D05938822029B52059B181B68DD
:1032A00008935A1C3CD044219AB20091402A04D879
:1032B0000320D11D814389B2009103991B0C8B42DD
:1032C00024D0402A22D80122300008A9FFF710FF9D
:1032D000021E1BD1380008A9FFF70AFF04000428CA
:1032E00031D9009A059B9B1880225201B218934253
:1032F00040D288235B05C118009A09A808F068FA33
:103300001D4B009A09A9F01808F0EAFA009A029BEE
:103310009446634402931A4B029AFB189A42BAD31A
:1033200088235B05FC1821680198013908F0A8FA88
:10333000200008F0E5FA039A07AB5A80300007999D
:10334000FFF706FF0400002C03D1002079E70428D2
:10335000FBD988235B05E018069908F091FA03234E
:10336000EA1C9A4300D16BE7034B0499E01808F07C
:10337000B7FA65E70424ECE704000011FFFFFF7FC4
:10338000F80F0000F7B505001400402A21D80027E7
:1033900001AE71803780FFF7FEFE042816D93A008F
:1033A0003100FFF7A5FE042810D93688BC420BD0A7
:1033B000BD4209D0221CB44200D9321C064B92B245
:1033C000C118280008F004FA30B2FEBDC04300B2B4
:1033D000FBE703204042F8E70400001137B5042260
:1033E00004000D0001A81649FFF7CCFF02000428D5
:1033F0000BD1019BA34208D3AB4204D0104901A8D2
:103400000195FFF7F9FE01203EBD0E4C2368200018
:10341000019308F075FA019920000139019108F033
:103420002FFA80235B01E418074B9C42EED1042263
:10343000034901A80195FFF7DFFE0020E4E7C0463D
:103440005555000000C007110000081130B589B0C3
:1034500008F006FA10226946254808F029FB254B9A
:10346000009A9A420ED1019B029A0F2B33D8002169
:1034700001240698013B08D2002900D00292029B49
:10348000013331D10023029325E0551CF2D1020013
:103490002100EFE710341022200004A908F008FBF7
:1034A000029B013301D1069B0293882304995B059B
:1034B000C918059B06981A03120B049105928142C4
:1034C00003D02B4201D108F083F9019B013B01930A
:1034D000019B002BDED1029B002B03D004930498A8
:1034E0004168084709B030BDE025014C2D03EFE7E6
:1034F00000000111504859368022F8B5964C974B80
:10350000D200002120001C6008F072FB2300944AC6
:1035100088331A60934B1A786A23002A00D011333B
:10352000E3620A232365904B37221B780820A363AC
:103530008E4B2118E361102323628D4B3B25636181
:10354000C823DB00A36123008C331A602823013ACF
:10355000E26320646364CA67043A211DCA672100DC
:10356000BC310D602100C03108602100C4310B6006
:1035700021000635CC310D602100083DC8310D60B9
:103580002100D0310A602200D43210602200D832EB
:10359000136022000227E032210017604222DC3152
:1035A0000A6021001B3DE4310D602100E831086014
:1035B0002100EC310B6023000521F4331960230056
:1035C000F0331A602300183290331A6023009433CA
:1035D000186023001E3A98331A60AF23DB00236083
:1035E000644BFA262363644B644DE360644BF03113
:1035F000A3642300FF31FC33B600A16021611E608B
:10360000A5627325E5656D3D6565A56596255D4AF1
:10361000AD00E264666258606766A566002709250A
:10362000A767E566584F594D606720002567E26738
:103630003A6015279C30676007001A203860200028
:10364000A0300700212038602000A83007004C4837
:1036500038602000F830066026006427A436376002
:1036600026005F3FAC3637602600033FB036376038
:103670002600C637B436376026000027B8363760D4
:1036800038269E60424E96205E64424E5A66DE6147
:10369000414E9A645E62F53EFF3E9E621E269A6728
:1036A000354A8000DE661F675F67DD651D6618624C
:1036B000DA67BE23394A5B00E250394BD8382350D1
:1036C00004302250C4225200A350C623E4205B00E1
:1036D000E1500433334AE1503349344BD16034492B
:1036E000800019503349E938FF3819503249043005
:1036F000195032493248D16132491163324951631C
:103700001900F4310860CE20304940001160304982
:10371000195019002F48F83108602F49D1658221CE
:103720002E4A89005A501A002D490832D1671A00D2
:103730002C49B432116088212B4A89005A501A0052
:103740002A49883211602A4ADA6408F0D1F8012047
:1037500007F0FEFFF8BDC0460004FF1F4464FF1FD2
:10376000106FFF1F1844FF1F4A0AFF1F3A0700008F
:1037700080C3C9019A020000DC0500006A1800003D
:1037800050C3000088130000F009FF1F204E000006
:103790006509FF1F68100000C409000040420F00C7
:1037A00010270000FC00FF1F751CFF1F0000FF1FFB
:1037B000C92CFF1F5130FF1FE92EFF1F3520FF1FAF
:1037C0002527FF1F5120FF1FFD21FF1FC11FFF1FC6
:1037D0004929FF1F312AFF1F8D19FF1F5528FF1F81
:1037E0007925FF1F8525FF1FC11EFF1F791FFF1FA2
:1037F000391EFF1F0223F0B50124624D624E2B706B
:10380000624B91B01C70624F039333680021082013
:10381000FB7006F001FE082006F0F8FC0023984239
:1038200005D0FA78552A02D0332A00D09DE03360C3
:10383000042006F06BFF07F0EBFEFFF75DFE08F0DB
:10384000FFF81F2201240021524B10AE1A70524B78
:103850001C70524B1970524B19689143163A0A4327
:103860001A60602219689143403A0A431A6008F0CE
:10387000DFF908F00DF94B4B9847C120FF214A4B67
:1038800080001A588A431A50C522920098588843DB
:10389000BF39014399509858444908408021C901D3
:1038A0000143802099509958C0050902090A014333
:1038B000995080213E48490108F072F80323220004
:1038C0003C49019400933C4807F0FAFF2C223B4905
:1038D00005A807F07DFF05AC61782078023406F07A
:1038E000B5FCA642F8D1364C0020012106F0C2FDFD
:1038F0002268344B03201A40A023DB0213432360C9
:10390000802322689B041343236022682E4B1A40B5
:1039100080239B03134323602C4A2D4B934200D8F2
:10392000012008F0D5F808F06BF980232268DB0449
:1039300013432360287808F00BF9039B1878C0B272
:1039400008F056F808F064F82249042008F0E0F87E
:1039500006F0A8FE00F040F800F0EAFD00F092FE4C
:1039600000F00CFA002011B0F0BD00932100194ABC
:10397000042008F0DDF88023DB059C62FFF766FD7C
:1039800056E7C0464A0AFF1F34F000401844FF1FA4
:10399000D861FF1F480AFF1F490AFF1F680AFF1F5F
:1039A000BCF00040E1A2000000E100E0FF00FFFFEA
:1039B0001C44FF1FA056FF1F1C54FF1F70BC0011AA
:1039C00014F00040FF7FF8FFFFFF9FFF0080FF1F04
:1039D000106FFF1F3B000108002210B511001120DD
:1039E00007F026FE10BD0000F8B500230926374F6A
:1039F000374C3B62E3681120B343E36007F0F8FE05
:103A0000112008F0ADF8112007F0B2FE4023226823
:103A100080251343236080236268DB0213436360C5
:103A2000A3682C4A2B43A360A36802211340A36020
:103A30008023A2689B0113431022A360236C0720FC
:103A400093432364236C0F3A1343236480235B0066
:103A50003B62226B204B1A402263626B1A40626306
:103A6000A26B1A40A263E26B1340E363E3681B4A54
:103A70001340E36006F0EAFB0121072006F0FAFCA0
:103A8000174B11205A6C15435D6407F059FFFD2157
:103A9000144B154A89005A508023C720626B5B0380
:103AA00013436363E36880003343E3600F4B104AC2
:103AB00019581140802212020A431A50802292059E
:103AC0001A6008220B4B5A63F8BDC04600F0004054
:103AD0003CF00040FFFFDFFFEFFFEFFFFFFF7FFF46
:103AE000003800400000FF1F5118FF1F00E100E0F8
:103AF000FF00FFFF0000054070B5284C238C002B11
:103B000023D0228A002A21D1DA0023826382A38271
:103B1000E38223836383A383E38322606260A260E2
:103B2000E2601F4D1F4A6420EB8093420AD8FA22BC
:103B30000020D200934205D91B4A0A21981807F0A9
:103B40001FFFC0B200232872238470BD0720E11C30
:103B5000CA7F01320240CA7705D10325201DC17FEB
:103B600001312940C17708325200A35200232100BD
:103B70001A00088A01321B180231082AF9D1221DC5
:103B8000D27F9200A350626823689B18A2689B189A
:103B9000E2689B185B099BB2C3E7C0461861FF1F30
:103BA000C061FF1FB70B000030F8FFFF30B503A85E
:103BB00004880B20002C0ED14968074D08784978FD
:103BC000090201430A20A94205D1012120001980E0
:103BD000024B1B7A137030BD192A0000C061FF1F11
:103BE000F7B5150008AA16884A680F4F147852785E
:103BF000120222430A24BA4214D10122DBB20192FA
:103C000000962A0007F09EFC041E0BD1074B1B6890
:103C1000002B07D068782A780002104342425041B6
:103C2000013098472000FEBD022900004461FF1FBB
:103C300030B5012503790400BFB02B4211D00A49E9
:103C4000408806F0EBFF28420BD0084B01A95B8DA2
:103C50004D800B80064B00221B7A60880B7104F0AC
:103C6000BDF83FB030BDC0463C61FF1F4840FF1F5C
:103C7000C061FF1F10B50549054806F085FF042106
:103C8000044A054806F042FF10BDC0463C61FF1FD4
:103C9000FFFF00009CBC00114840FF1F10B5024808
:103CA00004F01EFF10BDC046313C0011012303701B
:103CB0000B4B1A7A4270022282709A78C270DA78BC
:103CC0000271032242711A7982715A79C2710C22EF
:103CD00002729A794272DB7983720B207047C04678
:103CE000C061FF1F022310B50370013B4370053311
:103CF000837010330371443B43712A33837144331F
:103D0000C37100230372064B04001B8843720A3000
:103D1000FFF7CCFF831D0A30C0B2E37010BDC04670
:103D2000C061FF1F10B5142007F0D2FC124B142203
:103D30000021186007F05CFF002007F031FF012030
:103D400007F0C6FD022007F043FE032004F06CF9E3
:103D5000042006F081F9052003F0AAFB062004F0F8
:103D600077F8072001F06AFA082006F0AFFE092074
:103D700001F036F810BDC0464861FF1F07F0B8FCDF
:103D8000012007F06DFC07F0BBFC0000094B10B5EB
:103D90000400984205D0012904D12000064906F00C
:103DA000F3FE10BD0229FCD1013904F057FE0028B2
:103DB000F3D0F6E7FEFF00006E61FF1F70B50D7ACD
:103DC000100004AA2C00168810221440154220D19D
:103DD000002E20D10A78022A18D14A685178157825
:103DE0000E4A09022943914205D00D4A914209D059
:103DF0001C800A2404E014220A491A8007F0E8FC17
:103E0000200070BD0C2208491A80F7E71C800124AD
:103E1000F6E70824F4E70B24F2E7C046F3FF0000BE
:103E2000F4FF0000A442FF1F7CBD001110B5040088
:103E30000749084806F0A8FE074804F091FD002055
:103E4000E40704D50721054A054806F05FFE10BDCA
:103E50006E61FF1FFFFF00008D3D0011E0BC0011EF
:103E60008C40FF1F00B50C4BBFB01A780B4902A85D
:103E700000F0C2FC6B4680B2D880002809D06A46A8
:103E8000074B01A91B889380064B0022188803F07A
:103E9000A5FF3FB000BDC0464C61FF1F4D61FF1F35
:103EA000E640FF1FF041FF1F00B50C4BBFB01A7872
:103EB0000B4902A801F0D8FE6B4680B2D8800028DA
:103EC00009D06A46074B01A95B8D9380064B0022FF
:103ED000188803F083FF3FB000BDC0467661FF1F26
:103EE0007761FF1F8C40FF1FF041FF1FF7B50E00E9
:103EF000377A1C0008AB11003D001A8820231D40B2
:103F00001F423CD13378022B3BD173681F785B781A
:103F10001B023B431E4FBB4208D01E4FBB4214D076
:103F20001D4DAB4221D00A252800FEBD002A2AD112
:103F3000142C2AD82200F06807F04AFC174B1C709A
:103F4000012CF1D9FFF7B0FFEEE7002A1BD1202C9E
:103F50001BD82200F06807F03BFC114B04211C70B9
:103F6000104B187807F08CFDDEE7E3B201240092D5
:103F700001940A00310007F0E5FA0500D4E70825AE
:103F8000D2E70125D0E70B25CEE70D25CCE7C046CB
:103F9000F3FF0000F4FF0000022900007661FF1F1C
:103FA0004C61FF1FF861FF1F332310B5040003703D
:103FB0000A220749013007F00BFC064B0F201B6853
:103FC0001A0AE37222731A0C1B0E6273A37310BDDC
:103FD000C061FF1FE861FF1F30B5012503790400B0
:103FE000BFB02B4213D00B49408806F017FE284281
:103FF0000DD06A46084B02A81B889380FFF7D4FFB8
:104000006B46D8800022608801A903F0E7FE3FB02C
:1040100030BDC0466E61FF1FE640FF1F10B502486D
:1040200004F05EFD10BDC046D93F001170B516000A
:1040300004AA148805AA15784A68507811780002F5
:104040002A4A0843801805284BD807F0B1FD03130E
:104050001E29343F0720042C0BD80522121BAA422C
:1040600000D92A0022491A803000091907F0B0FB54
:10407000002070BD0720112CFBD81222121BAA426F
:1040800000D92A001B491A80EEE707200E2CF0D831
:104090000F22121BAA4200D92A0017491A80E3E70F
:1040A0000720032CE5D80422121BAA4200D92A00BB
:1040B00012491A80D8E70720032CDAD80422121BF1
:1040C000AA4200D92A000E491A80CDE70720032C06
:1040D000CFD80422121BAA4200D92A0009491A800B
:1040E000C2E700220A201A80C3E7C046DCD5FFFFE2
:1040F0002BBD00119461FF1F1BBD001116BD0011E7
:1041000011BD00110CBD001110B50D21024A03486C
:1041100006F0FCFC10BDC04600BD0011FC40FF1FB6
:10412000F0B50024274E85B03000B47100F0E2F8FD
:10413000254D264BEA89297C9A422FD10423300051
:1041400003AA00F057F90400300000F011F9012330
:10415000B371002C34D16B4699892B68C9BA4B4393
:1041600029891B4A1B145B1853806B46D9896B68DD
:1041700049BA89B24B4369891B0C5B181548191C55
:104180001BB2834200DD011C0B0400D50021138803
:10419000918001331380200005B0F0BD022722007A
:1041A00003AB3000009700F0F7F80E230400297CE1
:1041B0000122300000976B4400F0EEF80443C3E79F
:1041C0001C00E8E7D441FF1FA861FF1F8305000022
:1041D000C061FF1F0F27000073B5234E300000F0B1
:1041E00089F8224D07236A463000297C00F002F945
:1041F00004003000002C33D16B461B787F2B2FD866
:1042000000F0B6F86B46D878F02302041B031A407E
:104210006B469B8816495BBA9BB21A432B68000910
:1042200053432A891B0C9B184B806B465A789B780A
:1042300012031B011A436B68024353436A891B0C28
:104240009B180C481A1C1BB2834200DD021C13048D
:1042500000D500220B888A8001330B80200076BDB8
:1042600000F086F80124F9E7D441FF1FA861FF1F81
:10427000C061FF1F0F27000070B5114C237C002B7D
:104280000FD0382B0ED10F4D280000F033F8CC237F
:10429000AC222800217C9B0100F0F4F8280000F0FB
:1042A00067F870BD084BE2899A42FAD1054D2800A3
:1042B00000F020F800222800217C00F0C5F8EDE78E
:1042C000A861FF1FD441FF1F8305000010B5084BF4
:1042D0001A7C002A09D05B69002B06D09847041E7F
:1042E00001D0FEF78DFE200010BD0124F9E7C04685
:1042F000A861FF1F70B5C17905000C00631E9C41C9
:104300001A4BE402E41849000460C9B2007906F0CF
:10431000E7F8E979687949000131C9B206F0E0F8B7
:10432000E8790930C0B207F023FA0023E36661336D
:104330002360AA795B3B002A0ED022689A43023B95
:10434000134323600A23E3610733236200232363BB
:10435000A3630133E36370BD22689A4302231343CE
:104360002360462363610633A361EFE700500040FA
:1043700070B5002504000368DD66C0790930C0B25D
:1043800007F036FA2900207906F046F8290060790E
:1043900006F042F870BD0000F8B51E0006AB1D78AF
:1043A000002304681700E366616007F059FA0123EF
:1043B0008022E3662B0027615200013B08D207F000
:1043C000CFFA08200A4A1168002D03D12800F8BD51
:1043D0002261F2E7236F034203D02369013D33706A
:1043E000013613685B1A032BEED90125EEE7C046B0
:1043F0006008FF1F70B51C00002305681600EB66FF
:10440000696007F02DFA01238022EB662300520039
:10441000013B08D207F0A4FA08200A4A1168002CD0
:1044200003D1200070BD2A61F2E72B6F034203D055
:104430002B69013C3370013613685B1A032BEED9EC
:104440000124EEE76008FF1F002370B50468150023
:10445000E366616007F004FA0123E366256107F073
:104460007FFA8020064A80001168636B034205D101
:1044700013685B1A032BF8D9012070BD0020FCE7FC
:104480006008FF1F70B51D00002304681600E36676
:10449000616007F0E5F90123E36626610F33626B83
:1044A0001A42FCD02B0A23611023626B1A42FCD003
:1044B000EDB2256107F054FA8020074A80001168A8
:1044C000636B034205D113685B1A032BF8D90120F3
:1044D00070BD0020FCE7C0466008FF1F70B51E00DD
:1044E000002305681400EB66696007F0B9F9012341
:1044F000A619EB660F33B4420ED107F031FA8020D3
:104500000A4A800011686B6B03420CD113685B1A76
:10451000032BF8D9012070BD21782961696B1942FC
:10452000FCD00134E7E70020F5E7C0466008FF1F34
:1045300010B5084CE368002B08D18022064B5202CC
:104540001B689B186360054B1B68236007F078F8B5
:10455000A06010BDE861FF1FC8F00040CCF0004033
:1045600070B5184A936A916A9942FBD116498A68D4
:104570009A421FD39A1A8B60144B0126186893B283
:10458000D202D20E4343424300204C681B0A1B193F
:1045900012029B180E4C0A684B60551CA3420CD8A3
:1045A000002801D04B600A600A4A136008680A4B71
:1045B000186070BD581E821ADDE7084A30009B184B
:1045C0002A00EAE700F00040E861FF1F140AFF1F1D
:1045D00040420F00C8F00040CCF00040C0BDF0FFEA
:1045E00070B51F4C23793F2B01D93F2323711D4BFD
:1045F00022791A701878C0B207F022FB18231A49E2
:104600001A4A0B801A4913800B805380A3791949E9
:1046100080200B800C21938001334B43164D191CD5
:104620000001834200D9011C2980D1806379002BCD
:1046300011D101336371237A012B01D80223237234
:104640006279237A0D4853430A21584307F098F9B9
:104650000B4D286070BDA02BEDD9A023EAE7C04622
:10466000DC61FF1F480AFF1FEE41FF1FC443FF1F0D
:10467000EC41FF1FEA41FF1FE841FF1F71020000EC
:10468000CC61FF1FF8B514210020FEF7A7FE114CE6
:10469000011E114D09D10C22104BC1CBC1C4280001
:1046A00007F0A6FAFFF79CFFF8BD0C2220000C498A
:1046B000FEF768FE0C2802D0084B43CB43C40C2203
:1046C00028000849FEF75EFE0C28EBD00C220021E2
:1046D000E5E7C046DC61FF1FA861FF1F70BD001148
:1046E000FC0C0000F50C0000F0B51D4C8022A54428
:1046F0000400882069465201400507F029F99022FC
:1047000012016A441300200032C832C316C816C30F
:104710008023144C144FA6689B033343A3603B6073
:1047200007F0BEF98823A0685B05C01807F0E8F819
:104730000025882329008022A0685B05C018401945
:104740006944520007F0CCF880230135FF355B0146
:104750009D42EED1A6603E60044B9D44F0BDC04634
:10476000FCEFFFFF3443FF1F9808FF1F04100000F9
:10477000F0B5040087B0002825D0684606F068FF31
:104780001B4C022806D106226946200007F048F893
:10479000002816D06946002301250F262F00E25C71
:1047A000013310091030874038002F003240974005
:1047B0003A0002434A610439062BEFD16846FFF7FD
:1047C00093FF07B0F0BD182269460A4807F0C0F809
:1047D0006A46A300D358013305D01822FF2168464A
:1047E00007F006FAEAE70134062CF1D1E9E7C04602
:1047F0006509FF1F00090011F0B5002504000E0037
:1048000085B0AA4200D186E04B1C087801934B7812
:104810008978377909021943F3783F061B040B4363
:104820001F43039720706570252800D196E033D888
:10483000112813D807F014F9690025012501250175
:104840002501AA00B800B100250125012501250197
:10485000250125012501250105011F01232800D17E
:10486000DEE0DB2800D02EE1042A00D8ACE01025E1
:10487000052A05D0551F2A003800711D06F0A8FF33
:1048800005223100200006F0A3FF2A003900601D38
:1048900006F09EFF05353EE0562859D010D8332843
:1048A00000D19DE0552839D02628DAD19C4B29002B
:1048B000132218001D0007F09BF9FEF7A1FB5CE036
:1048C000712800D177E0722800D180E0602800D103
:1048D0008BE0DC28C5D1022A00D875E07378BFB21E
:1048E0006370B378A370032A05D0033A390092B2FB
:1048F000F01CFEF781FC10223900E01CFEF742FD9F
:10490000C51C002807DA60705CE00C222000854995
:1049100006F05EFF0C25280005B0F0BD013A824D7F
:104920000C2A13D8002A0AD02800019906F050FF5B
:10493000FFF756FE0C2228007C49FEF75DFC29009B
:104940000C22601C06F044FF0D25E4E70C22EBE787
:10495000754D774B2A0043CB43C2E9E7013A704DCE
:104960000C2A11D8002A08D00199280006F030FF3F
:104970000C2228006F49FEF73FFC29001322601C1F
:1049800006F026FF1425C6E70C22EDE705226A494A
:10499000601C06F01DFF0625BDE712226749601C5A
:1049A00006F016FF1325B6E708226549601C06F0DD
:1049B0000FFF0925AFE77178F02905D8614B1888FA
:1049C00001F0AEFD0225A6E7FF236370FAE75E4B18
:1049D000012A03D072789A706270F3E79B78F4E74B
:1049E0002000FFF7E1FA050095E7013A564B574DD5
:1049F000062A10D8002A10D00121280059700199E8
:104A000006F0E6FE01F05EF829000622601C06F0C2
:104A1000DFFE07257FE70622EEE700225A70F3E764
:104A2000042A04D94A4D2F6006F00AFEA860FFF759
:104A300097FD0422039003A9601C06F0C9FE05251A
:104A400069E7444D062ADFD906222800019906F0BD
:104A5000E7FE0028D8D006220199280006F0B8FE0B
:104A600006223D492800FEF7C7FB0123364A91780C
:104A70000B439370C8E7012AA6D07078FFF778FE41
:104A8000A0E7012800D0ECE6931E344F132B04D886
:104A90007378002B09D100F015F9314B39001D78DE
:104AA000601C6A1E06F094FE35E7551E2A00019927
:104AB000380006F08DFE2B49AAB23800FEF79CFBA9
:104AC00000F038F9E9E7DA281DD1042A00D87BE79D
:104AD000082A15D9B37972791B021343F2791204AB
:104AE0001A43337A1B0613433B603B6805223100AF
:104AF0002000039306F06CFE0422601D03A956E714
:104B0000FE236370F1E7DE2800D05DE7511E012A25
:104B100001D10025FFE6019800F0BAFFF9E7C04691
:104B2000A861FF1F7CBD0011DC61FF1FFC0C0000B1
:104B300070BD0011F50C0000B461FF1F9461FF1FF0
:104B40003843FF1FF041FF1FD861FF1F9442FF1F32
:104B5000E861FF1F6509FF1FADAC0000D963FF1FAF
:104B6000D763FF1FAEDE000070477047020010B52C
:104B7000094B0A32094C92B2DA815A829881188222
:104B8000207802F033FB0422054B012120781A70B3
:104B900006F076FF10BDC046C242FF1F2264FF1F11
:104BA0002164FF1F013870B5042809D807F000F808
:104BB000030928081200234B0221187806F060FF31
:104BC00070BD204B0821187806F052FE00221E4BC3
:104BD0001A72F5E7802200241B4B1A4D52001A81ED
:104BE00008211A682878DC7206F09AFF21002878DC
:104BF00006F076FD012000F083FE00F063FFDFE7A2
:104C0000104B0821187806F033FE1048FFF76AF8B9
:104C10000F4B104A9B79002093800F4A138080220B
:104C2000094B5200D8721A8100F06AFE00F04AFF68
:104C30000A4B9B78002BC3D0094A136006F068FD2D
:104C4000BEE7C046F861FF1FCC61FF1FF941FF1F9F
:104C5000DC61FF1FC443FF1FEA41FF1FD861FF1F34
:104C600034F0004010B501290BD1082809D1054BBB
:104C70001B78002B05D02622034B04485A72FFF7FD
:104C800075FF10BDFA63FF1FCC61FF1FC409000050
:104C90000300F0B50A4D8E18B14202D152008018BF
:104CA000F0BD0C782F6824093C5D0F271C700C7830
:104CB00001313C402F683C5D5C700233ECE7C0463C
:104CC000E441FF1F0E22124B10B51A700D23114C38
:104CD00011492370093A043B1048637006F078FDCF
:104CE0002D2301220E490F48E371FFF7D1FF012266
:104CF0000D49FFF7CDFF01220C49FFF7C9FF030063
:104D000000200B4902001870FEF776FA10BDC0466D
:104D1000F663FF1FD763FF1F2BBD0011D963FF1F71
:104D20006709FF1FDF63FF1F6609FF1F6509FF1F7C
:104D3000AEDE000070B5124C142220001149FEF7BF
:104D400021FB431E104D132B17D8AB78002B14D02A
:104D5000431C2B7009236B70002300190370287803
:104D600029000130C0B206F05BFC2978220001392D
:104D7000C9B2002005F0E8FD70BDFFF7A3FFEEE724
:104D8000D963FF1FAEDE0000D763FF1F10B5114BC4
:104D90001A781870002A0ED000280BD10E4B1A7802
:104DA000062A07D85423D340DB0703D50B4B1878CA
:104DB00002F01CFA10BD0028FCD0074B1B78012B19
:104DC00002D0033B022BF5D8044B0121187806F0E2
:104DD00057FEEFE7FA63FF1F2164FF1F2264FF1FE6
:104DE00070B5514E514A52493070082005F038FCD8
:104DF0000121022005F03EFB022005F01FFC0121ED
:104E0000002005F037FB002005F018FC00F0C8FE7C
:104E1000FEF7F6F806F00CFD032246494648FFF778
:104E200037FF2D24030004221C7044490130FFF792
:104E30002FFF30230470424D424C437083702E3B51
:104E4000062220004049EB87FEF79CFA062813D083
:104E5000200006F0FDFB022809D00321200006F007
:104E6000AFFC8D23E3706E3B23711933637106220F
:104E700020003549FEF7C0F9344B1B68FC335C64F5
:104E8000FFF758FF0020FFF781FF314C314A012125
:104E9000314B1278207802F06BF9304A304B12789F
:104EA0000021207802F064F901222E4B1A702E4B5B
:104EB000DB78552B31D12D4B3B325A722C4B2D4A7E
:104EC000AB81EA812B826A822021307806F088FE4D
:104ED0000120404205F084FD0120404205F020FE03
:104EE000FFF712F9FEF7C6FE00F0B2FC01204042C7
:104EF000FEF79CFF012006F0DBFCF02001F0F4FA45
:104F00000121307806F0BCFD307802F0CBFA1A4867
:104F100006F09EFEFEF768FD70BD6422174B5B79BC
:104F200053431A000A32CBE7F861FF1F694B0011A7
:104F3000654C00113843FF1F9461FF1FB461FF1FD0
:104F4000C242FF1F6509FF1FADAC00004464FF1F94
:104F50002264FF1F1842FF1FF941FF1FF663FF1F66
:104F6000D763FF1FC863FF1FD861FF1FCC61FF1FFE
:104F7000C4090000CE090000FA61FF1FDC61FF1FB9
:104F8000F8B50A0020230D001A40194263D05E4B89
:104F90001B78002B5CD0FFF7E3FA5C4B5C4C5D4E5A
:104FA00099686268737A8A1ADB039A4202D3616055
:104FB000FEF71AFD327A217A531EDBB2994205D1EF
:104FC000FFF75AF9002000F0B3FD15E09142F9D344
:104FD00000272772FFF77AF9A37ABB4202D0A772A3
:104FE000FEF78AFD012000F0A3FD4B4F3800FEF7CD
:104FF00079FE390006F0B4FB637A002B25D0013B23
:10500000DBB26372002B20D1444BDB78552B01D1EE
:1050100006F07EFBE37A002B12D00023A27AE37223
:105020009A4202D0A372FEF767FD3D4A3A4F1388B9
:10503000380001331380FEF755FE390006F090FB6F
:10504000642370795843FFF791FD237A013323726B
:1050500020206840F8BD0BB2002B0ADA314B1878DB
:1050600006F0D6FB002801D006F012FB80200002DB
:10507000EFE70224214206D0254B01201A72FFF7E8
:1050800085FE2000E5E70B071ED5FFF769FA1F4BE9
:105090001F49204C98684A68637A821ADB039A4257
:1050A00002D34860FEF7A0FCFFF710F9FFF7E4F821
:1050B000012000F03DFD00F0E5FB2368DB0701D592
:1050C000FEF7ACFF0820C4E7CB0609D5FEF714FDB8
:1050D0000D4B1B78002B01D1FEF7E0FD1020B8E747
:1050E0000124214207D0104800F06CF806F0B0FC13
:1050F00000F004FDC5E70424080020402142A9D0A7
:10510000FEF7B0FEBDE7C046FA63FF1FE861FF1F70
:10511000CC61FF1FDC61FF1FF941FF1FD861FF1F3A
:10512000C061FF1FF861FF1FDC41FF1FF0B51B4B83
:105130001B4F1B883A8804001A4E1B4D85B09A42BB
:105140000DD832889A420AD3184B1A882B889A4273
:1051500005D1174A174B12881B889A421BD005208D
:1051600001F018FA3B8802AA13803388019053801B
:105170002B88114D93800F4B02A91B88D3800F4BB6
:105180002A78188802F034FF0D4B08212878019AFC
:105190001C7006F0C5FA05B0F0BDC046C663FF1F1F
:1051A000EE41FF1FEC41FF1FEA41FF1FC463FF1FD9
:1051B000C263FF1FE841FF1F2264FF1FF041FF1F72
:1051C000C063FF1F13B50C4B1C78002C11D10028B5
:1051D00001D00A4B18600A4A0A4B11780A4A107823
:1051E0000A4A01920A4A0092002205F0A5FA20001C
:1051F00016BD1124FBE7C0462164FF1FBC63FF1FDF
:105200002064FF1F1064FF1F2264FF1FFC63FF1F49
:105210000064FF1F10B5064B12201B78052B06D12A
:10522000044B13221988044B187801F08FFB10BD32
:105230002164FF1FF041FF1F2264FF1F10B50024EF
:105240000122114B52421870104B1C70104B1A80E7
:1052500002F028F904220F4B21001A700E480C327C
:1052600006F0BEFB102221000C4806F0B9FB072215
:105270000B4B1C600B4B1C700B4B1C700B4B1A70B8
:105280000B4B1C7010BDC0462264FF1F2164FF1F22
:10529000F041FF1F2064FF1F1064FF1F0064FF1F09
:1052A000FC63FF1FD663FF1FD563FF1FF241FF1F83
:1052B000D463FF1FF8B5174C0600257806A8142400
:1052C0000078052D23D1B41F134FA5B21824BD4279
:1052D0001DD88D1FADB2BD4219D8FA256D00AA4266
:1052E00015D21D000D4F0A3DADB2BD420FD80C4C7A
:1052F00026800C4C21800C4900240A800B4A138024
:10530000FFF714FF0A4B0421187806F0B1FA2000C9
:10531000F8BDC0462164FF1F790C0000750C000029
:10532000EE41FF1FEC41FF1FEA41FF1FE841FF1F55
:105330002264FF1FF0B50BB20D0089B0002B00DB1B
:1053400070E1A44E307806F063FA041E50D0037862
:10535000A22B00D122E1D02B1AD0912B45D143783A
:105360000E2B42D19C4B82889A423ED19B4A836845
:105370001278052A39D1032018567F2835D0984B4A
:105380001B68002B31D05B68002B2ED098472CE097
:105390008078072829D806F00BFC0428183F3F74B2
:1053A000A8D86378002B0CD101218C4B19708D4B40
:1053B0001A78002A5BD08C4B307801F0D9FE002897
:1053C00055D00722854B1A7051E061780029F8D139
:1053D000E378002B11D0854A854B1278307801F0A4
:1053E000C7FE60706378002BEBD1200006F050F907
:1053F00080200002684009B0F0BD784B1B78022B7A
:10540000F3D00121307806F0D3F90028EAD1012148
:10541000307806F035FBE5E76378002BD1D16F4F8C
:10542000032807D13B78052B02D101333B701EE0E6
:105430000223FBE76F4B1A886F4B0293002A0BD0B5
:105440001B78002B03D00121307806F069F93B78F6
:10545000062B04D1013BE9E7029B1A70F7E7042B06
:1054600041D10121029B3078197006F009FB5C4B99
:105470001B68002BB9D01B68002BB6D0574A107898
:1054800084E76378554F002B27D10622211D5B4806
:1054900006F09EF962895A4B5A491A80A2895A4BE2
:1054A0001A80E3890B800521397058490A80584ACF
:1054B0001380228A574B1A80574B1B78012B09D136
:1054C0001F2001F067F8FA2292004243042130784D
:1054D00006F026F90022484B75E7312B00D070E723
:1054E0000022454B1A700323A0E7062200214348FF
:1054F00006F076FA0023454A04211380444A3078A6
:105500001380444A138006F0B3F90821307806F07E
:10551000AFF9A379083B5A425341304A0333137021
:10552000304B1B78002B06D0334B30781A78002A8A
:1055300006D001F05BFE0122314B52421A8096E701
:105540000121197006F09CFAF5E70821307806F081
:105550008FF96378002B00D047E72C4B2D4F029337
:10556000E388029A04211380294B3078039323891E
:10557000039A138063893B8006F01AF9002800D053
:1055800033E7264B1B68002B00D12EE703990298C6
:105590003A88098800881B68984726E74379132BC7
:1055A00000D022E70389012B0AD11D4B1B78022B67
:1055B00006D10821307806F05BF9FFF72BFE14E7DF
:1055C000052000F0E7FF08210200307806F0A8F877
:1055D0000BE7C0462264FF1F051400002164FF1F73
:1055E000BC63FF1F1842FF1FF941FF1FF663FF1F37
:1055F000D763FF1FF863FF1FFA63FF1FC963FF1F15
:10560000F041FF1FD063FF1FD263FF1FC663FF1F60
:10561000C463FF1FC263FF1FC863FF1FB863FF1F80
:10562000C063FF1F8020C001014200D0E2E6CB072B
:1056300031D5324B1B78002B1DD0314E05AC337861
:10564000052B1AD1023B23702E4B21001B782372AD
:105650002D4B1B7863722D4B187801F02DFD00281F
:1056600009D007202A4B30701B68002B03D01B6821
:10567000002B00D098470120BCE60E20254B0622C7
:105680001B7825492370254B1B78637002ABC0182B
:1056900006F09EF8D8E7022308001840194209D006
:1056A000174B1B78052B03D11D4B188806F028FAE1
:1056B00002209FE60424214203D0FFF737FD20009B
:1056C00098E6082308001840194200D193E6154BCC
:1056D0001C78012C03D0022C0DD008208AE6124B36
:1056E000124A134913481B881288098800880094BD
:1056F000FFF7E0FDF1E7FFF78DFDEEE7FA63FF1F2F
:105700002164FF1FF241FF1FD463FF1F2264FF1FAC
:10571000BC63FF1FD663FF1FF341FF1FD563FF1F4D
:10572000F041FF1FC063FF1FE841FF1FEA41FF1F59
:10573000EC41FF1FEE41FF1F10B502A804880B20AB
:10574000002C10D1496808784978090201430C48B7
:10575000814209D1022119800A4B59881170DB78E6
:1057600000205BB2537010BD074C0A20A142FAD151
:1057700002211980034B998811705B79F0E7C046CC
:105780006E2A0000C061FF1F6F2A0000F7B51500E8
:1057900008AA16884A680F4F1478527812022243DA
:1057A0000A24BA4214D10122DBB2019200962A00E7
:1057B00005F0C8FE041E0BD1074B1B68002B07D059
:1057C00068782A78000210434242504101309847DD
:1057D0002000FEBD022900003464FF1F30B5012502
:1057E00003790400BFB02B4225D01449408805F04E
:1057F00015FA28420CD0124B01A95B8D00220B80B8
:1058000002234B800F4B5B888B80608802F0E6FAA6
:105810000D49608805F002FAC0070CD50B4B01A9B1
:105820001B8800220B8002234B80064B9B888B80B9
:10583000608802F0D3FA3FB030BDC0462C64FF1F31
:105840001C42FF1FC061FF1F2464FF1F7642FF1F21
:1058500010B5074C0749200005F096F920000649CD
:1058600005F092F90721054A054805F04FF910BDEA
:10587000FFFF00002C64FF1F2464FF1F9CBD00116C
:105880001C42FF1F10B5024803F02AF910BDC046A4
:10589000DD57001170B540253F2608210B4BC2078C
:1058A000D2172A40DD789C7835408C432A439C707F
:1058B000DA70820701D521439970400704D5802210
:1058C000D97852420A43DA7070BDC0469442FF1F35
:1058D00013210A4BDA788A43123901400A43DA70FD
:1058E0000222104202D0D9780A43DA70400703D569
:1058F0001022D9780A43DA707047C0469442FF1FDD
:1059000010B5054B082419790A00A243002801D0DC
:1059100022000A431A7110BD9442FF1F10B5054BB7
:105920002024D9780A00A243002801D022000A438B
:10593000DA7010BD9442FF1F0821F8B5324D334B89
:10594000AE7804000E40AE70984204DD67232B70E1
:10595000273B6B70F8BD2E4B984203DAE0232B7087
:105960001A3BF6E700232B706B7083B21A002948AC
:105970005F3292B2284F82422CD9002C03DA5B426C
:105980001CB204232B70053420B20A2105F0F8FF65
:1059900004B2FA239B009C4232DB08232A7813438B
:1059A0002B706421200005F0EBFF0A2100B205F006
:1059B000EFFF09B22A787B5C13432B700A21200089
:1059C00005F0DEFF0A2100B205F0E2FF09B27B5CC0
:1059D0006A780AE06970002CDBDA5B421CB20423AF
:1059E0002B70F5226B78092CE8DC13436B700A21CD
:1059F000200005F0CDFF09B27B5C1E43AE70A9E725
:105A0000632CCEDCEDE7C0469442FF1F1B4E000026
:105A10001DFCFFFF2A080000C7BD00110823F7B5D1
:105A2000194FCD003E7904001E403E71EDB263284F
:105A300006DD5F3333433B7140231D437D71F7BD6A
:105A40000300093305DA20235B4233433B71C6234D
:105A5000F3E70E4B019300280BDA0423444224B2EF
:105A60003B710A21200005F093FF019B09B25B5CAA
:105A7000E3E70928F5DD0A2105F082FF019B00B26A
:105A80001B5C1E433E71ECE79442FF1FC7BD001133
:105A9000F8B50A4F05003B780E00002B0CD0084CDF
:105AA0002000FEF727FC33002A0020003978FEF79B
:105AB00015FD2000FEF75CFCF8BDC0463864FF1FF2
:105AC0009C42FF1F70B50A4E0A4D06223100280085
:105AD00005F0A6FE002809D0074C31000622280058
:105AE00005F076FE07212000FFF7D2FF70BDC0460B
:105AF0009442FF1F8E42FF1F8D42FF1FE62220218E
:105B000010B50A4B1A70203A5A701C329A70DA7823
:105B10000A40DA70082219791140033A0A431A71CF
:105B200027225A71FFF7CEFF10BDC0469442FF1FD7
:105B300070B5184B5C78002C2BD1002829D0164D5D
:105B40000A210223E85E05F01BFF00B2FFF7F4FE16
:105B50000423E85E642105F013FF012100B2FFF782
:105B60005DFF132220002B7A9A426041C0B2FFF7FA
:105B7000D5FE0320FFF78EFE2000FFF7A9FE074B9E
:105B80001878053843425841C0B2FFF7B9FEFFF715
:105B900099FF70BDD861FF1FC061FF1F2164FF1F07
:105BA00070B500250A4C2000A571FEF7A3FB112358
:105BB0003E212000074AFEF791FCA84200D13E3565
:105BC000054B20001D700123A371FEF7D1FB70BDB2
:105BD0009C42FF1FB6BD00113864FF1F0200F0B5E4
:105BE00001270A480A4E51188B1A002B00DCF0BD21
:105BF000082415784308684038404000805B013C29
:105C000058406D08002CF5D10132EDE7FFFF000090
:105C1000D8BD0011F0B500250F269D4200DBF0BD78
:105C20004C5D070944403440A400A0580135784039
:105C3000F3E70000F0B589B06A460D000B000F27AE
:105C4000110010351C780133260024093E401670DF
:105C500054700232AB42F5D12023024AFFF7DAFF3B
:105C600009B0F0BDDCBD0011F0B54E780B7889B0FD
:105C700036020C00170001901E43012A61D9954B92
:105C80009E4200D877E001339E421CD1062A17D1EC
:105C9000CA788B7812021A430B791B0413434A7992
:105CA00012061A438C4B5A6100221A705A808B4A92
:105CB0005A608B4A9A608B4ADA60002009B0F0BDC6
:105CC00088225205EEE7884B9E423CD182498B7870
:105CD000002B00D0F6E00C2A31D10F22A378934399
:105CE000E2781202134322791204134362791206F6
:105CF00013434B60E279A07912020243207A000438
:105D00001043627A12060243CA60E27AA07A120253
:105D1000024376484A81834208D804236E491422FC
:105D200001980B7005F054FD1420C7E71201D2183A
:105D300089235B059A42F0D801238B70BDE7022AC4
:105D4000FAD00523EAE76A4A01239642E6D1FFF733
:105D500061FA052F0CD9E378A2781B02134322794C
:105D600012041A4363791B061343624A03931360B8
:105D700005F0CEFCA1E7584D2B78002B9DD1AB78D8
:105D8000002B00D1A0E02B8901339BB20093B342DA
:105D900000D091E0132AD4D9CF7C8B7C3F02122112
:105DA00020001F43FFF71AFF874200D08EE0002E2D
:105DB0003DD1E378A2781B0213432279E9681204EB
:105DC0001A4363791B06134303930A228B4212D1B1
:105DD000FF23A370E370237163716B89002B09D1DA
:105DE000E37B227C1B0212041343A27B13431B0997
:105DF00001336B8100226B89002B8ED0002A67D182
:105E0000686837013818000B6B69000303909842EB
:105E100005D9686105F074FDEB780133EB706868B3
:105E20001022A11C381805F05BFD2E8145E76F8913
:105E3000009A7B1E9BB293423AD1E278A378120279
:105E40001A43237905A81B04134362796C68120670
:105E50001A43EB6800920392211D0C22049305F073
:105E6000B7FC0120260004A940421036FFF7E2FEED
:105E7000013F012F17D1009A0B232861824200D0E5
:105E80004CE704221C49200005F02AFD042203A946
:105E9000686805F05DFDE968039AFF23914200D12F
:105EA0003CE7F73B3AE73100FFF7C4FE1036DFE787
:105EB0000923B742A4D831E7009BB34200D9FCE6DE
:105EC00007232BE7022329E7032327E7062325E7F8
:105ED0000A2323E7FFFE0000A442FF1F0000011178
:105EE000FFFF00005048593601FF0000FFFF00117E
:105EF00002FF000034F00040B042FF1F10B5034C19
:105F00000B000122210000F06BFA10BDBD600011F2
:105F10000B8870B506000D000224162B11D92B003A
:105F20000322094900F05CFA041E0AD1074B2A88B3
:105F30001B88191C934200D9111C300089B200F053
:105F4000EFFA200070BDC046E96000114A64FF1FEF
:105F500010B54A780400013A0B000220012A07D844
:105F60000A78002A04D005222000024900F038FAFD
:105F700010BDC046176100110A7810B50B0004006F
:105F80000220002A04D007222000024900F028FA4B
:105F900010BDC046C36100110A7810B50B000400A3
:105FA0000220002A04D009222000024900F018FA39
:105FB00010BDC0462962001110B5034C0B000B2226
:105FC000210000F00DFA10BD5962001110B5034C0C
:105FD0000B000D22210000F003FA10BDCB6200116E
:105FE00010B5034C0B000F22210000F0F9F910BD91
:105FF000256300110A7810B50B0004000220002A66
:1060000004D011222000024900F0EAF910BDC04678
:1060100035630011002310B51322190000F0E0F9D8
:1060200010BD000010B5034C0B001722210000F03A
:10603000D7F910BD87630011002310B5192219008C
:1060400000F0CEF910BD000010B5034C0B001B2270
:10605000210000F0C5F910BDC1630011F7B58489B6
:106060000D0006000121002C22D000238268D356A7
:106070001778002B1EDA0C2C1AD90C3CA4B2131979
:1060800040880093230002F086FE431E98410130B1
:106090007B06DB0F6B703F23013C1F40A4B22870CE
:1060A000AF70AC80002C07D0B3680133AB60002127
:1060B0000800FEBD0020EBE7AC60F8E70B7803704A
:1060C0004B8843704B881B0A83700B79C370042084
:1060D00070470420022B06D10020537811781B0250
:1060E000009A0B43138070470B8803700B881B0AC0
:1060F0004370022070470420009983420AD15378EC
:1061000010781B0203430B80D37890781B02034363
:1061100000204B807047F8B50D004B78012400211A
:10612000461C03702B788B4201D82000F8BD6B7899
:10613000B01C4F1C012B10D1890069184B8802221A
:1061400033704B88B9001B0A7370691805F058FC4E
:1061500004360434A4B2F9B2E4E7122359436B18AD
:106160005A88043132705B8810221B0A73706918D8
:1061700005F046FC12361234ECE770B5049D1400AD
:106180001E00052B01D8042070BD637812781B0215
:1061900013432B80E378A2781B02134302226B8007
:1061A0002A71211D681D063E05F02AFCB2B22A8123
:1061B000E92AE8D82800A11D0A3005F021FC0020BA
:1061C000E2E7002310B50A789A4201D8900010BD8A
:1061D0009A008A185488013304705488DBB2240A68
:1061E0004470948884709288120AC2700430EAE77E
:1061F00010B51100029C062B04D004201022142B91
:1062000001D010BD022222714B7808781B02034393
:106210002380CB7888781B02034363800431601DA0
:1062200005F0EEFB0020ECE710B50C788B7804311C
:106230005C43E4B203702200013005F0E1FB601C16
:1062400010BD0420022B06D10020537811781B02C8
:10625000009A0B431380704710B50C000A88023176
:1062600005F0CEFB208810BD70B504000D00049829
:106270001100012B01D8042070BD1678527812024B
:10628000324302800200F13255701470E125002C77
:1062900000D10C35023B9AB24280AA42EBD80231BF
:1062A000043005F0ADFB0020E6E7042000998342AE
:1062B0000AD1537810781B0203430B80D37890786F
:1062C0001B02034300204B80704710B50C000A8866
:1062D000023105F095FB208810BD000070B501214A
:1062E0001E000420049C0E400B4218D1CB40DDB2AE
:1062F0008D4214D90A49DBB2098899420FD3230091
:10630000EE331D703300580011184978165C0902ED
:10631000314301332152D9B28D42F4D8002070BDEF
:10632000BC42FF1F10B50C000A88023105F068FB63
:10633000208810BD10B50C788B7804315C43E4B232
:1063400003702200013005F05BFB601C10BD10B52E
:1063500011000298032B01D8042010BD1478527844
:10636000043B120222430280CA788C781202224334
:1063700042809AB28280EB2AEED80431063005F0D2
:106380003FFB0020E9E710B50C000B8803700B8879
:106390001B0A43704B8883704B881B0AC3708A8822
:1063A0000430063105F02CFBA088043080B210BD0B
:1063B0000420012B03D100201378009A137070473A
:1063C00010B50C000B8803700B881B0A43704A88B9
:1063D0000230043105F014FB6088023080B210BD39
:1063E000F0B589B003931E4B029242000700D05AC9
:1063F000019102F020F81325061E2DD0029B0124E6
:106400000370019B002B04D00019039998470019D1
:1064100084B26B461B7A5BB2002B0FDA1021380076
:1064200002F01CFB1925002813D130003219E1B20B
:1064300002F066FC051E0CD10C34A4B2042304AA9D
:10644000380005A993800696948101F0AFFD051EE2
:1064500002D0300005F074F9280009B0F0BDC04644
:106460004864FF1F70B505000C0000280CD0002008
:10647000814209D010222000044905F0C1FA012010
:106480002B7823736B78637370BDC0461CBE0011FC
:10649000F0B506000D0017001C0085B002291BD0C6
:1064A0000020102907D1022B07D0102B03D115E0B3
:1064B0000020102C08D005B0F0BD69463800FFF769
:1064C000D1FF2A0069460BE069463000FFF7CAFF9A
:1064D00022006946380004E0022BE9D12A00390085
:1064E000300005F02DFBE6E7031CF02800D9F0236F
:1064F000032008499AB2013A0B80D317034006499A
:106500009B189B100B80D30F04499B185B100B80CA
:106510007047C046C042FF1FBE42FF1FBC42FF1F64
:10652000034B1B888B4202D3024B4000C152704781
:10653000C042FF1F4864FF1F014B4000185A7047BC
:106540004864FF1F1722014B1A8070474864FF1FE1
:1065500070B505000E2005F013F9041E13D0D023EA
:10656000037000230622837007494570033005F04D
:1065700047FA064B2100DA8A62811B7E2373044BA3
:10658000187805F015FA70BD6464FF1F5464FF1F8E
:106590001043FF1F262803D8024B4000C05A704703
:1065A0000148FCE7C242FF1FFFFF000070B5060074
:1065B0000C00094D1C220021280005F011FA074BA0
:1065C0001E70074B1C7005F01BF90123002801D039
:1065D000002312202B7070BD5464FF1F1043FF1F57
:1065E0007564FF1F70B505000D4C0800E260A160E6
:1065F00010220021656005F033FB012803D1102132
:10660000A06802F058FD10220021280005F028FBA8
:10661000012803D11021606802F04DFD70BDC04615
:106620005464FF1F70B5041E05D1002903D0062253
:106630000D4805F0E5F90D4B1D78012D11D1002C09
:1066400005D102221A7005F0FBF8280070BD002267
:106650001A70074B1B78FF2BF7D02000FFF778FF4D
:10666000F3E70025F1E7C0466464FF1F5464FF1F91
:106670001043FF1F030010B5002801D1002010BDFA
:1066800000780B4A002803D15988D1821B791376F0
:106690001378022BF2D10023984200D103331370F8
:1066A000044B1B78FF2B01D0FFF752FF0120E6E7D8
:1066B0005464FF1F1043FF1F002911D000280CD085
:1066C0004B79012803D140225242134303E03F2279
:1066D0001340032802D001204B7170474022F4E799
:1066E0000800FAE770B5094D0100287800280BD0A2
:1066F000074C0622200005F083F921002878FFF7D7
:10670000DBFF200005F064FA70BDC0467464FF1F13
:106710004E64FF1F00290AD0012808D13F224B797F
:106720009343C02B03D0403B5A425341981C7047BF
:1067300070B5174D06002B78FF2B15D00A2005F0F9
:106740001FF8041E10D0D0230370C83B8370114B78
:1067500011491B784670C3700622043005F050F9C9
:106760002100287805F024F90C4B1B78012B0DD162
:106770000B4B1B68002B03D09B68002B00D0984765
:10678000084B04211878084A05F0CAF970BDC046C4
:106790001043FF1F7464FF1F4E64FF1F7064FF1FD0
:1067A0009C64FF1FA064FF1F60EA0000014B986813
:1067B0007047C0465464FF1F014BDB681868704780
:1067C0005464FF1F074B10B5DA6813680133136078
:1067D000054B1878FF2803D08021C90105F050F936
:1067E00010BDC0465464FF1F1043FF1FF7B50E00D5
:1067F00002F0C8F8051E1CD00E4B06621F78002F51
:1068000000D10778AB791020019304F0B9FF041E82
:106810000FD0D0230380C73B8370019BE91DC37059
:106820000622043005F0ECF821003800E66005F09F
:10683000BFF8F7BD0E43FF1F014B18787047C046E5
:106840007464FF1F054B002805D1054B1A78054BD2
:10685000002A00D1014B18007047C0466464FF1F36
:106860007464FF1F4E64FF1F014B58687047C04699
:106870005464FF1F024B1868431E9841C0B2704712
:106880007864FF1F421E03000120152A03D9FF3B35
:106890005A425341D8B27047F0B51C0000230E0095
:1068A00085B0039002920B70029A934201D30020AC
:1068B00019E0E55C5A1CD2B2002DF8D002985119AB
:1068C0008142F4DC0233DFB2A35C18000193FFF7CE
:1068D000D9FF002807D0013D019A0399EBB233702C
:1068E0008A4202D1E01905B0F0BDDB19DBB2DBE76B
:1068F00010B50C0002F09EF803001220002B03D00C
:106900002100588804F0B4FE10BD000070B50E4D93
:1069100084006359002B15D0186A002801D004F0B8
:10692000CFFE2B59586A002801D004F0C9FE2B591C
:10693000986A002801D004F0C3FE285904F0C0FE74
:1069400000232B5170BDC0468464FF1F1C4B70B5E3
:1069500004000E00150099420AD11A4B1B68002B47
:1069600001D1122070BD1B68002BFAD09847F9E7BF
:10697000154B994215D1134B1B68002B0AD01B688D
:10698000002B07D09847002804D1104B1C70104BE7
:106990001D70E7E729002000FFF7AAFF0028E1D1DA
:1069A000F3E7080001F0EEFF0028DAD003780320B7
:1069B000A342D7D12900300004F05AFED2E7C046E6
:1069C000FEFF00008064FF1FFFFF00007D64FF1FCB
:1069D0007C64FF1FF7B50400808801F0D3FF002519
:1069E000A84203D00578A08802F008F81C4E33783E
:1069F000002B1FD0AB421DD11A4B28001978FFF78E
:106A000077FF002818D000233370A3790820A778D7
:106A1000A688019304F0B4FE011E0DD0D0230370AC
:106A2000CA3B8370019B477086808371280004F005
:106A3000BFFF01E0002DE8D1A0880B4B8200D358A6
:106A4000002B01D0FFF762FF1721A088FFF768FD38
:106A5000A08801F027FDA08801F0FEFDF7BDC0462B
:106A60007D64FF1F7C64FF1F8464FF1FF0B587B047
:106A70001D000CAB1B88070001930DAB1B88142075
:106A800002930EAB1B88160003930FAB1B8800917B
:106A9000049310AB1B88059304F072FE041E1AD0F9
:106AA000D0230370CB3B47708370C6700622290049
:106AB0000430002D11D004F0A3FF019B210063815D
:106AC000029B0098A381039BE381049B2382059B87
:106AD000A37404F06DFF07B0F0BD04F081FFECE794
:106AE000F7B5009308AB1B8807000C200D001600BB
:106AF000019304F045FE041E13D0280001F042FF6C
:106B000000280FD00078D0232370C93BA370009BCE
:106B100021002381019B6770A580E680638104F0DA
:106B200047FFF7BD014B1878EDE7C0461043FF1F44
:106B300013B5040064890389C2888188C0780094F1
:106B4000FFF7CEFF13BD000010B5044C20680028ED
:106B500003D004F0B5FD0023236010BD8864FF1F3F
:106B6000A122F0B5818892004A43384B384F1B6808
:106B700004009B189D2292009B18827989B01A60AC
:106B80003B68002B5FD01D78324B1B68002B04D074
:106B90005B68002B01D000209847260008363100A2
:106BA000E079FFF7B7FD237DE0710200E078049300
:106BB000638A29000393238A0293E3890193A388BC
:106BC00000933300FFF752FFE378002B0BD1E289EB
:106BD000A379A18802920196E2792800009201220D
:106BE00001F0DAFEE0703B68002B20D0FFF7ACFF2D
:106BF000194D287800281AD0184B1978FFF778FE1D
:106C0000002814D02B78E67808200793A78804F092
:106C1000B7FD011E09D0D0230370CA3B46708370B4
:106C200087808671079804F0C3FE00232B7017211C
:106C3000A088FFF775FCA08801F034FCA08801F063
:106C40000BFD09B0F0BD064B9DE7C0463409FF1FA0
:106C50008864FF1F9C64FF1F7D64FF1F7C64FF1F0F
:106C60001043FF1FF8B5070008000E0001F08AFE70
:106C7000041E18D02620FFF78DFC051E00D12578B4
:106C8000062004F07DFD041E0DD00021062204F034
:106C9000A7FED0232370C23B21006770A370A6809B
:106CA000E8B204F085FEF8BDF0B585B001930AABFB
:106CB0001B78070002930BAB1B7808000D000092B5
:106CC000039301F05FFE061E22D0102004F058FD51
:106CD000041E1DD01022002104F082FE2620FFF7A2
:106CE00059FC002800D13078D0232370C13BA37019
:106CF000009B21002372019B67706372029BA58039
:106D0000A372039BC0B2E3720C9BE36004F050FEDD
:106D100005B0F0BDF7B50D00019001F033FE071E80
:106D200020D00E2004F02CFD041E1BD02620FFF7DF
:106D300031FC061E00D13E78D0232380C53B0622BD
:106D4000A370F91DE01C04F05BFE019B2A00638127
:106D50000123DD401A401D40210022736573F0B20B
:106D600004F026FEF7BD0000F0B585B002901000DB
:106D70000D0017000A9E039301F004FE041E31D09B
:106D8000029B002B2ED1039B02795B0724D5122393
:106D900013430422002E08D10B99002905D10C9928
:106DA000002902D10D9900291AD01A430D9B227196
:106DB000002B00D0C9E0002E00D1CFE0002D00D084
:106DC000CCE0606A002801D004F07AFC1C2130007D
:106DD00004F066FD606205E002239A430E33D7E7B4
:106DE00093432371654BBA00D458002C00D1AAE01C
:106DF000002E10D0236A002B03D11C2004F068FC65
:106E000020625E4BBA00D358186A002803D01C22B7
:106E1000310004F0F5FD0C9B002B12D0574CBB0049
:106E20001D596B6A002B03D1162004F051FC6862D7
:106E3000BB00E358586A002803D016220C9904F0CE
:106E4000DFFD0D9B002B11D04C4DBC006659B36A81
:106E5000002B03D1142004F03BFCB0622B59986A3C
:106E6000002803D014220D9904F0CAFD380001F067
:106E700089FD051E67D0414BBA00D358002B62D064
:106E80001A6A3420002A00D11C389A6A002A01D0DC
:106E9000143080B20B9A002A01D01C3080B25B6A99
:106EA000002B01D0163080B204F06AFC041E4AD0D8
:106EB0001822002104F094FD2620FFF76BFB0190BF
:106EC000002801D12B780193D0232370029B20004E
:106ED00063700A23294EA370039BBD00A371AB59B5
:106EE000A780196A1830002905D01C22A06004F080
:106EF00087FD200034307359996A002907D00300B8
:106F000014221433E060029304F07AFD02980B9B84
:106F1000002B08D003001C221C330B992061029324
:106F200004F06EFD02987359596A002903D01622A5
:106F3000606104F065FD6B462100187904F038FDAE
:106F40003800FFF7E3FC05B0F0BD10220D9B0D9952
:106F50001B69A018236204F053FD2CE70B9B002B48
:106F600000D13FE7012D00D03CE7606A002801D046
:106F700004F0A6FB1C210B982AE7C0468464FF1F7F
:106F800010B5044C2068002803D004F099FB0023BE
:106F9000236010BD7864FF1F0B4B07B51A68002AE9
:106FA00001D100200EBD6946531C01201278073123
:106FB000FFF772FC0028F4D002780123100018407B
:106FC0001A42EED0EEE7C0469464FF1FF0B51F4FA3
:106FD00001203B6887B0002B25D09B78059300F0FB
:106FE000B3FB002821D00A20FFF7D4FA04000B20BD
:106FF000FFF7D0FA164B05001E78731E9E413B68C2
:10700000F6B2191DD878FFF757FB3B682900DA7AEA
:10701000043303929A790193029200903300200086
:10702000059A04F0CDFD07B0F0BDFFF7B5FF0028CD
:1070300005D00620FFF7AEFA04000720D8E70820A5
:10704000FFF7A8FA04000920D2E7C0467864FF1FC2
:107050007464FF1F70B50A4E040033780D00FF2BD7
:107060000DD0042004F08CFB011E08D0D023037047
:10707000CE3B45708370C470307804F099FC70BDCD
:107080002043FF1F70B5040006200D0004F078FBBC
:10709000011E0AD0D0230370CD3B8370054B447092
:1070A0001B688580187804F083FC002C01D0FFF762
:1070B00067FF70BD7864FF1FF8B5264F06003B6878
:1070C0000D001124002B05D10522234B1B78134200
:1070D00002D112242000F8BD204A10241268002A90
:1070E000F8D01278002AF5D0DB0719D52B789A1E34
:1070F000012A1AD80C2004F0EBFA13243860002877
:10710000E8D000230A22437029000670023004F000
:1071100077FCFFF75BFF041E0AD0FFF731FFD9E7CA
:1071200000F012FB0028E1D1E4E7002BE2D0D0E729
:107130000B4B1B78032BCDD11D20FFF72BFA094BEE
:1071400018800028C6D0084B04211878074A04F09C
:10715000E7FCBFE77864FF1F7564FF1F9464FF1F9F
:107160007464FF1F7264FF1FA064FF1F60EA0000C9
:10717000F7B50193194B14001A78052306000F0088
:1071800012201A4221D0012920D1154B1D68002D53
:107190001BD002201F2C18D8002C02D0019B002BE2
:1071A00013D0104B1F221E706E1C0021300004F003
:1071B00017FC01992200300004F022FC310020006D
:1071C0002C70002F06D004F0ABFBFEBD064B122046
:1071D0001D68DCE704F024FAF7E7C0467564FF1F7A
:1071E0009464FF1F2043FF1F9064FF1FF8B50F4EEC
:1071F00012243368002B17D01B780F3C834213D125
:1072000000250B4F0221387804F032FB094B042192
:1072100038781D8004F02CFB074B28001D80336854
:107220005C7004F0FDFB04002000F8BD7864FF1FD3
:10723000A064FF1F8C64FF1F7264FF1F70B50128DC
:1072400023D11B4C2388002B03D01A4A1578002D1C
:1072500007D0194B1B68002B02D01878FFF7C6FF28
:1072600070BD3B2B02D93C3B2380F9E7134E022132
:10727000307804F0FDFAFA222388920002215A4362
:10728000307804F04DFA2580EAE70B4B1B68002BA1
:10729000E6D00B4B1B785B07E2D5084B0221187830
:1072A00004F0E6FA0022024B1A80FFF769FED7E7E6
:1072B0008C64FF1F7064FF1F7864FF1FA064FF1FB2
:1072C0007564FF1FF8B51E4D2868002803D004F030
:1072D000F7F900232B601B4E3068002803D004F020
:1072E000EFF900233360184F05243B781800204045
:1072F000234221D0154800F02BFA3B78234213D0CB
:10730000202004F0E5F92860002813D02022002175
:1073100004F066FB202004F0DBF9041E306005D089
:107320002022002104F05CFB002004E0286804F027
:10733000C7F92C601320F8BD00F00AFAF4E7C04644
:107340009464FF1F9064FF1F7564FF1F1443FF1FA9
:1073500010B50A4C23681A1E0ED0002808D101303F
:10736000587004F05DFB002805D02368002B02D084
:107370000021FFF787FE0122100010BD7864FF1F77
:10738000F7B5274E050033680191181E21D05C78AF
:10739000244F012C30D1FFF7FFFD002825D020001D
:1073A000FFF7F8F80400412814D91F4B0221187880
:1073B0001E4A04F0B5FB1E4B3C3C1C800222336885
:1073C0005A703B78002B14D128000199FFF75AFE20
:1073D0000120FEBDFA2292004243002AEED0124B59
:1073E0000221187804F09CF9E8E7FFF7D3F80200CF
:1073F000F3E700233B70EBE73B78002BE8D1032059
:1074000004F0BEF9011E08D0D0230370CC3B4570B8
:1074100083703368187804F0CBFAFFF7B1FDD7E733
:107420007864FF1F7064FF1FA064FF1F60EA000004
:107430008C64FF1F10B51749838802008B4220D04F
:1074400011D815498B4217D0144900205B1899B206
:10745000012907D8926811785A425341D8B2FFF7F0
:10746000F9FD012010BD0E4A00209B1807229BB297
:107470009A424041C0B2F5E783681878FFF768FF89
:10748000F0E7836899785A78090218781143FFF772
:1074900077FFE7E70A20000006200000F8DFFFFF83
:1074A000AFDFFFFF014B18707047C0462143FF1F3D
:1074B00010B5064C207001F041FA207804F080FAF3
:1074C0000521207800F062FD10BDC046A064FF1FBA
:1074D0000BB273B50D00002B00DBC4E0884B1878AD
:1074E00004F096F9041E0ED00378912B0FD0A22B36
:1074F00000D1A1E0834B1878FF2852D0210004F07E
:1075000057FA00284DD180200002684076BD4378AC
:107510000F2B76D013D8052B70D00E2BEAD1808894
:10752000794B98422BD8794B98421BD8784B98428C
:10753000E0D1A3681878591CFFF774F838E03E2BA7
:10754000D8D18378032B74D06CD8012B6ED0022B4A
:10755000D0D1704B1B68002B23D05B68002B20D050
:1075600098471EE06C4BC0180C28C3D804F0B8FA3A
:107570001DC2C2150BC20B0B0B3223C23C00674B62
:10758000C0180728B6D8664B1B68002B09D01B68AB
:10759000002B06D0200098470AE0A3681878FFF770
:1075A000C7F8200004F074F8ADE7A068FFF762F8B0
:1075B00000289FD0F5E7A3681B78002BF1D0554B2E
:1075C0001B68002BEDD01B68002BEAD0210055482A
:1075D0009847EDE74F4B1B68002BE2D01B68002B50
:1075E000DFD021005048F3E7504B1B68002BD8D068
:1075F0005B68002BD5D021004348E9E7FFF7EAF9A3
:10760000CFE780884A4B984203D04A4B984200D03B
:1076100070E7464B1B68002BC3D05B68002BC0D0C3
:107620002100D5E7153B012BBBD963E7FFF798FA9B
:10763000B7E7FFF77DFAB4E73F4B1B78042B07D180
:1076400000236A4613800179408800F0C5FCA8E752
:10765000364B1B68002BA4D05B68002BA1D0010027
:10766000364898479DE7012421420AD0294B1B68E0
:10767000002B04D05B68002B01D00020984701202C
:1076800043E78B070AD5264B1B68002B04D05B68A9
:10769000002B01D020009847022036E70421280063
:1076A00008400D4200D131E7254E3388002B21D010
:1076B000013B9BB23380002B1AD1FFF7DBF8002887
:1076C0000AD0204B1C70164B1B68002B04D05B6843
:1076D000002B01D020009847FFF7C6F8694601F05B
:1076E00001FD6846FEF7FEFF1D20FEF753FF3080C8
:1076F00004200AE7024B187804F0BAF8F8E7C0460D
:10770000A064FF1F2143FF1F0E2000000120000086
:10771000091000009864FF1FFEDFFFFFAFDFFFFFCF
:107720009C64FF1F0C2000000B2000008064FF1FE2
:107730000D200000132000007564FF1FFFFF0000F4
:107740007264FF1F7064FF1F10B501F09BF910BD3C
:10775000014B18607047C0469C64FF1F0B880020D7
:10776000162B01D817230420014A13807047C04606
:107770004A64FF1F00207047074A030011888142B6
:1077800007D091880020994202D101308000101862
:1077900070470020FAE7C046A864FF1FF0B58F7855
:1077A00006000D00C5B01E2F15D1FFF7E5FF051E21
:1077B00003D10024200045B0F0BD00223B00310081
:1077C000C078009200F0B2FB0400A81C00F0D2FBCD
:1077D000FF23EB70EEE7264B062403931B78FF2B69
:1077E000E8D0182FE6D87B08224A013BDB00029242
:1077F0009A589446002ADDD0029AD3185B68002B71
:10780000D8D00878002802D14B78012B02D1062469
:10781000122FCFD107AFAB88697800976446AA686A
:10782000A047041EC6D1AB78029A5B08013BDB007F
:10783000D318390030005B689847041E0BD1AB7831
:10784000042BB6D0039A310010782200009700F084
:107850006DFB0400AEE76A78002AABD1AA7805A9CF
:107860003B88087130000A704B80FEF747FBA0E7A9
:107870002443FF1F2CBE00111D4B37B50500984255
:107880000BD000290AD1FFF777FF002805D119484E
:10789000FFF772FF002800D0058037BD01291AD1FB
:1078A000FFF76AFF041EF8D001235B420380A37830
:1078B000FF2BF2D0FE2B07D00023E0781422009398
:1078C00029001E3300F032FBA01C00F053FB012303
:1078D0005B426380E1E70229DFD1013901F0BEF8A4
:1078E0000028DAD12800FFF747FF041EDFD1D4E7D4
:1078F000FEFF0000FFFF0000022210B5074B5242BE
:107900001A80074801325A809A80DA8000F07EFAA5
:10791000044801F025F8002010BDC046A864FF1FF0
:107920009D770011797800110388F7B50400002BCA
:1079300002D102252800FEBD4268022113782548A5
:107940005268FEF7A5FD00282ED0234F01253A8866
:10795000002AEFD0802321885B0201259B1A9942DF
:10796000E8DC0C2003F0B4FE061E31D03B882288F0
:107970009C4600231800019561469DB2491989B2C1
:10798000AA421BD8002801D062443A80002330006C
:10799000082208C0210004F033F8104A1368002BB5
:1079A00013D100251660C5E76268022113780C48E0
:1079B0005268FEF76DFD0028C7D1BAE760681D0167
:1079C0004019418101330198D6E71A001B68E6E7A8
:1079D0001325AFE79ABE00112243FF1FA464FF1FC7
:1079E00098BE0011014B18707047C0462443FF1F1A
:1079F00014230A0010B51A40194204D001221021A4
:107A000001F048F810BD4B06F9D40120884340002E
:107A1000F8E710B514008B0604D50122102101F0FF
:107A200039F810BD08230A001A40194202D14BB29E
:107A3000002B0FDA102101F02DF8002808D02300C8
:107A4000F2331B78002BECD0F1342378012BE8D1F2
:107A50000020E6E703208907FAD4E2E7F0B51F002B
:107A6000184B85B01C68019002910392002C27D11D
:107A7000200005B0F0BDA5683301ED186B89019AAF
:107A8000934211D3029A93420ED8002F04D10A9B3D
:107A9000002B10D12C00EBE73B002978039A686893
:107AA000FEF7F6FC0028F2D10136B6B2A388B34245
:107AB000E1D82468DAE7A3680A9A5B891380E9E7CA
:107AC0000026F3E7A464FF1F37B50C000A88498835
:107AD0000123914217D3002A15D0651D23792A006E
:107AE00002210A48FEF7D4FC102300280BD023798A
:107AF0006188208800242A000094FFF7AFFF0A2342
:107B0000A04200D0230018003EBDC0469ABE00111E
:107B100013B50A0008884988012388420BD8002839
:107B200009D00024137905320094FFF797FF0A2348
:107B3000A04200D02300180016BD13B50A00088823
:107B40004988012388420BD8002809D000241379E2
:107B500005320094FFF782FF0A23A04200D02300E1
:107B6000180016BDF0B58BB003904A8808880E0047
:107B70000123824255D3002853D00023012704ACAF
:107B800023700022718813000092FFF767FF051E23
:107B90003ED02078002835D12B78022B18D1677081
:107BA0006A8983000130E31880005A8069680222E4
:107BB000201803F025FF23780133DBB22370042B58
:107BC00019D93B006889013080B2002BD9D01FE061
:107BD00002236370122358436A89231804305A80A1
:107BE00069681022201803F00BFF23780133DBB201
:107BF0002370002BE5D10C4A6B899B185A425341E4
:107C0000DBB2DFE76378012BE4D12B78022BC7D0FE
:107C100022780A23002A04D021000398FEF798F95D
:107C2000002318000BB0F0BD0100FFFF0F4BF0B5B3
:107C300004001868002816D083685D89A54207D81B
:107C40008288AE18B44203DA12019A18934201D125
:107C50000068EFE71E005F891036A74204D10029B3
:107C600000D00D801800F0BD3300EFE7A464FF1FC3
:107C700070B505000C0008880021FFF7D7FF03004E
:107C80000120002B04D022002800197AFFF7C1FE42
:107C900070BDF7B50C00002501902300EE331B7872
:107CA000AB4201D800200AE06B00E65A0021300008
:107CB000E718FFF7BBFF002802D126800130FEBD88
:107CC000017A0198FFF794FE002802D03B882380B8
:107CD000F5E70135EDB2E0E710B5040008880021B2
:107CE000FFF7A4FF03000120002B03D02000197A26
:107CF000FFF77EFE10BD0000054B1B68002B01D175
:107D0000180004E09A6852898242F6D19888704738
:107D1000A464FF1FF0B50E27002687B0039302ABC3
:107D2000FF183E8005001F4B40891400984207D081
:107D30002B78013000976A6880B2FFF78FFE06004B
:107D400002212B7818486A68FEF7A2FB00280FD0A2
:107D50006C892000FFF7D0FF002802D0013C0419F5
:107D6000A4B2039B002B00D01C80300007B0F0BDF4
:107D700002212B780D486A68FEF78AFB0028E7D1BC
:107D800002212B780A486A68FEF782FB002807D098
:107D9000002EDED03B88A342DBD17489013CDFE7B3
:107DA0006C89DEE7FFFF00009ABE001198BE00114B
:107DB00096BE001110B50C00FFF7DEFC0300022098
:107DC000002B0AD0002C00D023609B781720FE2BBC
:107DD00003D00138FF2B00D1002010BD73B50D007A
:107DE00001A904001600FFF7E5FF172805D0002EB3
:107DF00004D129002000FEF727F976BD01221021C9
:107E0000200000F047FE0028F3D0F6E7014B186091
:107E10007047C046B464FF1F37B56B469D1D010017
:107E200004000222280003F0D3FC2B88B02B0ED1D3
:107E30002379122B09D12300FA331B78012B06D1A9
:107E40000121608800F0E0F801E01B2BF8D037BD7D
:107E500010B5054B0421187000F098F8FFF74CFDA1
:107E6000FEF770FB10BDC046B864FF1F0020F0B5E0
:107E70000BB20F0087B0834234DA274B187803F037
:107E8000C7FC051E2BD00378A02B25D103AE3100F3
:107E9000FEF7E4F8041E0BD1B378DB0724D51F4BA3
:107EA00006341B68002B03D0310068889847040013
:107EB000A868002801D003F043FC002C08D1184A20
:107EC000039B1340174A934206D0B3781B2B03D071
:107ED0000121688800F098F8280003F0D9FB802081
:107EE0000002784007B0F0BD0F4B1B68002B10D08C
:107EF000310068889847041EDAD07378002BD7D1F8
:107F0000B27801A90A704B800C716888FDF7F6FF02
:107F1000CEE70624F1E7C046B864FF1FB064FF1F38
:107F200000FFFF0000011200B464FF1FF7B50190CD
:107F3000FC200D0017001E0003F022FC040013209B
:107F4000002C12D0B02320002370089BF42267700D
:107F5000658026710830002B08D0190003F050FD11
:107F60002100019803F024FD0020FEBD089903F0D4
:107F700037FDF5E710B5041E06D00078FD2803D8BC
:107F800003F086FCFF23237010BD00000A1F93B28C
:107F900010B504000220032B05D882400020024BBC
:107FA000D1529B189C7010BDD864FF1F0B8870B510
:107FB000043B04000D000220032B0BD801212000FC
:107FC00000F04CFD03001420002B03D029002000FA
:107FD00000F0DEFB70BD000007B51300034A0092FD
:107FE0000A00012100F02CFC0EBDC04615820011D4
:107FF00007B5019203220092024B0A00122100F001
:1080000049FC0EBD9382001107B56B4601AA118091
:108010000449D88008780633012802D1190003F0FA
:1080200087FC07BDB964FF1F0C4B10B51870002307
:10803000FF210B4A1380138193819380094A538057
:108040001370517293819372D174D38213755177E7
:1080500003F09EFD00F0FCF910BDC046E864FF1F70
:10806000D864FF1FBA64FF1FF0B58DB06B460020C7
:1080700003910C229B5E834200DBB0E05D4B1878DD
:1080800003F0C6FB051E00D1A4E00378902B00D0BE
:108090009DE006AF01004688380000F013FA7968C9
:1080A0000400002900D19CE03B88052B6ED13B8960
:1080B000032B1CD905AC200000F0A2F86288172A17
:1080C00061D83989131D994231D1796823780431F7
:1080D0000291D90738D5607800F08EF9071E06D0D6
:1080E000002303712378012B08D0132B23D0A86819
:1080F000002800D178E003F023FB75E06288029944
:1081000009A800F0A6F80290380000F08BF909AA3F
:108110002378387A0192002231000092029A00F00E
:1081200012F9380000F064F9029B002BDFD0300018
:1081300000F080F9DBE70378032BD8D1628802993D
:1081400009A800F0D6F8DEE7122B13D1029909A88E
:1081500000F0B5F8021EEAD127498B88002BC6D063
:10816000887909A92378019161780091310000F0A4
:10817000EAF8BCE7002302AA93833000617809AAD9
:10818000FFF72AFFB3E71D4B0993F6E7042B02D054
:108190009A1F012AABD8184A043B9B00995A002920
:1081A000A5D0D218907831003A0000F0AEF800283F
:1081B0009DD13B88042B03D001213000FFF724FF21
:1081C000012C04D1A868002801D003F0B9FA2800D6
:1081D00003F05EFA8020039B0002434018000DB0BC
:1081E000F0BD012800D182E701213000FFF70CFF2C
:1081F000EDE7C046E864FF1FD864FF1F01001700C9
:108200000B7803704B784370CB788A781B0213434A
:10821000438070470A88030002700A88120A42707D
:108220000A88012A06D14A8882704A88120AC270D6
:108230000420704702208242FBD14A8804309A70A1
:108240004A88120ADA708A881A718A88120A5A7160
:10825000EFE710B50400012082420CD94B780A7870
:108260001B0213432380834206D1CB788A781B02FA
:1082700013436380002010BD022BFBD1CB788A789A
:108280001B02134363804B790A791B021343A380BB
:10829000F0E70B8803700B881B0A43704B888370D0
:1082A0004B881B0AC3708B8803718B881B0A437130
:1082B000CB888371CB881B0AC371082070470300E9
:1082C0000120082A14D14A780878120202431A8041
:1082D000CA788878120202435A804A7908791202D1
:1082E00002439A80CA798879120202430020DA8018
:1082F000704710B504000120022A05D100204B78F8
:108300000A781B021343238010BDF8B50600102025
:108310000F00150003F034FA04000120002C0ED0E9
:10832000A0230C22290023806780201D002D07D068
:1083300003F066FB2100300003F03AFB0020F8BD9B
:1083400003F04EFBF6E7F7B51E00009008AB1420D3
:1083500017001D78019103F013FA041E12D0A22316
:108360000370019B47704380099B057146710C2285
:108370000830002B07D0190003F042FB21000098C1
:1083800003F016FBF7BD099903F02AFBF6E737B5B2
:10839000041E0FD04388002B0CD00025C188132366
:1083A000007A172201950095FFF7CDFFFF23658026
:1083B0006372257037BD000010B50C4904004A886F
:1083C000002A09D08B89002B05D00020CB8A0222FD
:1083D000834201D010BD012213000A204343002034
:1083E0004032C854C81842800472F3E7BA64FF1FD1
:1083F0000023438003707047094B00211A0010B519
:108400005C88002C06D01C79844203D10A234B439C
:10841000D01810BD01310A330329F1D10020F8E74B
:10842000BA64FF1F10B50400407A03F031FAFF234D
:10843000637210BD7047043010B580B203F058FB72
:10844000002803D00421494203F0CAF910BD0000FE
:1084500070B50025104CA0682580A581A580A84294
:1084600002D003F06DF9A56000250C4C0C4B606D3B
:108470001D80230058331D70A84202D003F060F91C
:10848000656500256068002801D003F059F90135C1
:1084900008340A2DF6D170BD8065FF1F2465FF1FCB
:1084A0007465FF1F70B5041E09D1054D2880A88191
:1084B000A880A868002802D003F042F9AC6070BD23
:1084C0008065FF1FF0B54B8885B0019300234360A2
:1084D0000A7905000F00022A00D07BE0CA88032A2F
:1084E00017D98B685E7819783602DC78D8790E4314
:1084F00099781B7A24021B020C43034353495BBA4D
:108500000B80331D93421ED1042C04D0631F022B19
:108510000ED9012015E0019A4D4B1201D35A002BC0
:1085200006D00198FFF7BEFF4A4A13690133136171
:108530000421B8682E812C80494203F051F968600B
:10854000002005B0F0BD434D042C06D0631F022B64
:108550000FD9EB680133EB60DBE7019A3C4B12016A
:10856000D35A002B05D00198FFF79CFF2B690133EC
:108570002B61374B30000293019B029A1B01019340
:10858000002301998C468B52130063449C80039313
:108590009E81FFF750FF039B041E986016D00421B4
:1085A000B868494203F01CF9FA880100043A200037
:1085B00003F026FA0199029AFB888A5A043B9B1819
:1085C000029A8B522B6801332B60A2E7AB6901330F
:1085D000AB619EE71E4B0293019B1E01029BF35A67
:1085E000002B2DD002998C19A068002828D0012AD0
:1085F00026D1FA889B189BB27352A189994217D34E
:108600009B1AC018B96803F0FBF9029BA289F35AC0
:10861000934200D07DE700222B81A3882B80A368A2
:108620006B60029BF2520B4A53680133536070E750
:10863000084A9368013393600198FFF733FF68E7B6
:10864000044A536901335361F6E7C046EA64FF1FE9
:108650008065FF1FF064FF1F70B5051E15D10B4C20
:108660000B4B1880230058331870606D002802D01F
:1086700003F066F86565250050356068002801D074
:1086800003F05EF80834AC42F7D170BD2465FF1FDB
:108690007465FF1FF0B51700A12285B09200019309
:1086A0004243394B06001B680C009B18D933FF333B
:1086B0001D78FDF741FF0430854204DD3000FDF7F1
:1086C0003BFF0430C5B2BD4207D33A000021300061
:1086D000019B03F04DF905B0F0BD2900380003F00F
:1086E0005FF82300C6B250331E700393019B29002C
:1086F0006365380003F0ACF8CBB20293002B02D0D4
:10870000039B01361E7000262300503303931B7811
:10871000B34204D8606D002831D10020DBE7029A13
:108720002800002A04D0013B1000B34200D02800EA
:10873000F700E719387003F073FA786000280ED05C
:108740003A78019903F05CF9019A3B780136D31825
:108750000E4A0193D369F6B20133D361D4E7039B88
:1087600018706065A74205D1084A1320D36A013307
:10877000D362B0E7606802F0E3FF0834F2E702F08A
:10878000DFFF00236365C8E73409FF1FF064FF1FA4
:10879000F7B50D0007000421686803F021F82B8964
:1087A000040003702B891B0A43702B8883702B886D
:1087B0001B0AC3702E8902250436F6B2F42E15D892
:1087C0001B4B9F4214D10C2002F0DAFF1135011E21
:1087D0000CD0902303708E3B0371043B4380154BF8
:1087E0008460C680187803F0E3F800252800FEBDF9
:1087F0005C237B43104AD3180093583301931B78B2
:10880000002B0FD10300320038000099FFF742FF20
:10881000019B05001B78002BE8D13800009903F07C
:1088200077F8E3E7054A0725536A01335362DDE72A
:10883000FEFF0000E864FF1F2465FF1FF064FF1FB8
:10884000F0B587B0009017200F0016000193FFF7D6
:10885000F2FD1325041E19D00C98031E02D00199B5
:10886000201D9847030AE370052302AAA070043074
:10887000908127700098667003A993800494FFF795
:1088800087FF051E02D0200002F05AFF280007B023
:10889000F0BD0000F0B587B01F000CAB1B78039152
:1088A000059301210DAB06001C78049200F0D6F868
:1088B0001425002821D02000FFF77EFD0135041E7D
:1088C0001BD01149059B0A7803700132D2B2131EE6
:1088D000C68001D101231A000B7022713000049B65
:1088E00003990097FFF7ACFF051E09D12300210073
:1088F0000648074A093303F09BF8280007B0F0BD8B
:10890000002363802370F8E7EC64FF1F8F8300115E
:1089100030750000F8B505000E00064C064F2368C0
:10892000002B02D03100280098470434BC42F6D115
:10893000F8BDC0469065FF1FA465FF1F0123064ACE
:108940005B425380002313715362044A13605360E7
:108950009360D36013617047A465FF1F9065FF1F8C
:108960000200002310B506499C000859002801D1D7
:10897000625010BD0133052BF6D11320F9E7C04634
:108980009065FF1F034A5388181A434258414042DA
:1089900010407047A465FF1FF0B585B002930AAB85
:1089A0001F780CAB1B88009008000E000192039307
:1089B000FFF7E8FF05001120002D1BD10E48FFF73F
:1089C000E1FF04001520002C14D006220B99A7719A
:1089D000E01D03F015F8019B30002371029B290074
:1089E0006371009B66802370039B6562E381FFF7E0
:1089F00091FF280005B0F0BDFFFF000010B5FFF7A4
:108A0000C1FF04000220002C12D060880121FFF772
:108A100081FF606A002801D002F052FE2822002166
:108A2000200002F0DDFF012300205B426380207103
:108A300010BD000030B5074A074C55880100137877
:108A40000020A54204D05B1A59424B4158421040C5
:108A500030BDC046A465FF1FFFFF0000084A10B5E7
:108A600001230C00904208D0FFF78CFF031E04D0B6
:108A7000037923405A1E9341DBB2180010BDC04653
:108A8000FEFF0000024B1879431E9841C0B27047A8
:108A9000A465FF1F70B504000D001600FFF772FFFC
:108AA000002804D10D4B9C4200D0143070BD416AA7
:108AB00003790520002907D012221A40102A02D17A
:108AC0000520002EF2D10F20DB06EFD5897E0C2089
:108AD000A9428941494249420840E7E7FEFF0000B8
:108AE000030010B5002800D110BD0348034A418897
:108AF0009142F9D09847F7E7A465FF1FFFFF0000F8
:108B0000002330B5C45CCD5C6C40D4540133102BD1
:108B1000F8D130BD0F23002210B5C45C640022439D
:108B2000CA54C25CD209013BF7D210BD0200010059
:108B300010B52032103102F0B3FD10BDF0B58BB08E
:108B40000390102005931700049102F0C1FD0090DE
:108B5000102002F0BDFD009B13240190002B05D0D6
:108B600000280CD11324009802F0AAFD019B002BD1
:108B700002D0180002F0A4FD20000BB0F0BD1020C0
:108B800002F0A6FD0600102002F0A2FD132405004D
:108B9000002E00D1AEE0002819D01022002102F0F2
:108BA0001FFF32002900039802F07AFD041E0ED147
:108BB00033787F2B51D830000099FFF7ABFF009B33
:108BC0001B787F2B53D801990098FFF7A3FF300043
:108BD00002F076FD002D02D0280002F071FD002C7D
:108BE000C1D1102002F074FD0600102002F070FDCB
:108BF0000290002E7CD0002878D03A000F3223005B
:108C00000125121105D00F333B4015B25A42534192
:108C10001BB26A1E1201002B33D0049BD2B29818EB
:108C20000099029AFFF76CFF013D102200213000ED
:108C300002F0D6FEADB2049F2D017D19AF4242D0A5
:108C4000002C33D0300002F03BFD029B002B00D102
:108C500089E7180002F034FD85E729003000FFF7AE
:108C600059FF28002549009AFFF74AFFA7E7290086
:108C70000098FFF74FFF28002049019AFFF740FFB7
:108C8000A5E70F210F4004998A18D9B28F4208D95D
:108C9000D15C06A819540133102BF6D1029A019920
:108CA000C0E7791A48424141C901F2E73900300072
:108CB00006AAFFF725FF3200039806A902F0F0FC90
:108CC00010370400BAE7002CBCD13000029906AA84
:108CD000FFF716FF320006A9039802F0E1FC082214
:108CE00004003100059802F08BFEABE71324A9E7DE
:108CF0001324AAE7002800D06EE733E7A0BE0011D6
:108D0000F0B58BB00F0016000225009000283FD070
:108D1000002A3DD00B1DDBB21800029302F0D8FCF4
:108D20001135041E34D0FDF747FD05003A000099C7
:108D3000201D02F0C5FEEBB20393E3702B0CDBB2F7
:108D40002F0A00936370FFB22B0E2370A77001935C
:108D5000FDF72CFD1022010006A802F0B1FE210053
:108D6000029A04AB06A8FFF7E9FE051E0DD1039B8E
:108D700008223370009B04A9B370019B7770F370D5
:108D8000301D02F09DFEFDF71DFD200002F098FC55
:108D900028000BB0F0BDF0B58FB00D00149E03900D
:108DA00004920593002A03D1022420000FB0F0BDE5
:108DB000002EF9D00398FFF7E5FD1424071EF4D028
:108DC0007278337812021A43B3781B041343F27893
:108DD00012061A43036A0192934201D30133E3D18D
:108DE000002D03D03B7901249B07DED5082200210A
:108DF00006A802F0F5FD059B13240433DBB218002E
:108E0000029302F065FC051ECFD0059A0499043048
:108E100002F056FE04223100280002F051FE390013
:108E2000102210310AA802F04BFE2900029A06AB6C
:108E30000AA8FFF783FE041E0FD1082206A908A87E
:108E400002F03EFE0822311D08A802F079FE01283A
:108E500007D101990398FDF7C9FC280002F030FC06
:108E6000A3E70124F9E7000070B51C4C0500236856
:108E7000181E10D0002D14D11A78002A0CD1981C7D
:108E8000083202F0BDFD02F073FE0135002808D162
:108E900023681D70012070BD0A331800082202F0FB
:108EA000AFFD2368002BF5D0122002F069FC061EEE
:108EB0000DD0C123216803704570023110220230A9
:108EC00002F09EFD23683100587802F071FD2068A1
:108ED00002F0F6FB00232360DCE7C046CC65FF1FF1
:108EE000F8B504002020FDF755FB0D4EA700BB5937
:108EF0000500002B0DD000280BD0D878FF2809D111
:108F000008492A000C55F35907480333611802F049
:108F10008FFDF8BD290002F0ABFD0028F0D1F8E785
:108F2000E865FF1FD065FF1F39A1001170B5064D20
:108F300084006359002B05D0D87802F0A9FCFF22E9
:108F40006359DA7070BDC046E865FF1F70B5060052
:108F50008CB00C00150000213022684602F040FD64
:108F600031001022684602F0ABFD1D2021000322D3
:108F7000684402F0A5FD6846FFF7D8FD2D210400E6
:108F800003222800694402F09BFD20000CB070BD54
:108F9000F0B50700160097B001931CAB1D78302286
:108FA0001EAB00910AA800211C7802F019FD1022C6
:108FB00039000AA802F084FD1022002102A802F064
:108FC0000FFD0722310002A802F07AFD072202AB52
:108FD0009818631E9C41019902F072FD02AB9C73CC
:108FE0002B005A1E934102AAD3730021102206A817
:108FF00002F0F6FC06221D9907A802F061FD1A2076
:1090000002ABC01806221F9902F05AFD10220099E7
:109010000EA802F055FD102202AB0EA908781C78AC
:10902000013A6040D2B2087001330131002AF5D113
:109030000AA8FFF77BFD102212A904000EA802F077
:10904000DFFC102206AB0EA908781D78013A6840B3
:10905000D2B2087001330131002AF5D10AA8FFF716
:1090600065FD044310222098E4B212A902F028FD05
:10907000200017B0F0BD70B50E0014008CB00100D8
:10908000102268461D0002F01BFD3100082204A8D2
:1090900002F016FD2100082206A802F011FD684624
:1090A000FFF744FD04001022280008A902F008FD83
:1090B00020000CB070BDF8B506000D000024371973
:1090C000AC4200D3F8BD02F063FB030A3B70631CA3
:1090D000DBB201379D4203D90234F054E4B2EEE72B
:1090E0001C00EDE773B506000C000225002819D01E
:1090F000002917D0032101A8FFF7DDFF6B469A79FD
:109100003F231A40013313436A463000937101A98B
:109110002200FFF71BFF051E04D10322E01C01A95A
:1091200002F06EFC280076BD03785807DA08C00FFD
:10913000D20080009B0710439B0F1843C0B27047BA
:1091400007230B40C908C9000B4303707047000098
:1091500070B50400FFF7EAFE134DA4006359002B1D
:1091600021D0186A002801D002F0AAFA2B59986E73
:10917000002801D002F0A4FA2B59D86E002801D0A3
:1091800002F09EFA2B59186F002801D002F098FACD
:109190002B59586F002801D002F092FA285902F09A
:1091A0008FFA00232B5170BDE865FF1F0E4B800026
:1091B000C35870B50C00002B0FD09D68002D0CD04B
:1091C0002B78201D0B706B784B70A97CFFF7B8FFD4
:1091D0002B7E23726B69E36070BD1022002120009A
:1091E00002F0FEFBF8E7C046E865FF1F014B186080
:1091F0007047C046E465FF1F074A0300800082589D
:1092000010B5002A06D0D088984203D1012901D197
:10921000FFF79EFF10BDC046E865FF1FF0B5264E64
:1092200095B087000B93BB590500099112200A9253
:10923000002B31D0D888FFF7A5FB04001420002CA8
:109240002AD0280010A9FFF7B1FFBB591E781D6A6C
:10925000002E23D00895FDF7EFFA07000020FDF758
:10926000F1FA0790A379E61D069310AD0CA90898B2
:1092700000F0E2FA0EA9280000F0D7FA0B9B0A9939
:109280000493069B09980293079B0396019300970A
:109290000EAB0CAAFFF77CFE15B0F0BDFDF7CCFAC3
:1092A00006903000FDF7CEFAE31DA779079310ABC7
:1092B00006000893DAE7C046E865FF1F30B50C4C9E
:1092C00085002A59030085B00120002A0ED018001D
:1092D0006946FFF76BFF2B591A78D888054B002A8F
:1092E00000D1054B6A46072100F0D9FB05B030BD1F
:1092F000E865FF1F2B9800113998001130B5094C13
:109300008500295985B010226846253102F078FB86
:109310002A591121044BD0886A4600F0C0FB05B0E1
:1093200030BDC046E865FF1FD598001130B5094C27
:109330008500295985B010226846353102F060FB5E
:109340002A591121044BD0886A4600F0A8FB05B0C9
:1093500030BDC046E865FF1F13990011F7B54D4FAA
:1093600086001020F4590D0002F0B2F9F359206282
:10937000186A132200286CD0033A29009C6802F076
:109380003FFBF3591A780192002A58D11E6A227DB8
:10939000317B944651400122019F114201D1674621
:1093A0001740217D914339432175377B4F40BC469F
:1093B00060460027800701D44F0817400121022092
:1093C0008F40227D82433A432275377B5740BC460B
:1093D00060460027400701D497080F400420227DF3
:1093E000BF0082433A432275627D0027944660465F
:1093F000727B42400A4201D167460F400121627DE3
:109400008A433A436275777B5740BC4660460027E3
:10941000800701D457080F400220627D7F008243FD
:1094200017436775767B00227E40760701D4BA0821
:109430000A400426617D9200B1430A4362756A784E
:10944000002A08D06278002A05D005220533DA7791
:1094500000221000FEBD04222979114205D1A17C11
:10946000114202D10533033AF1E7019A21782C78B1
:10947000002A02D10A002100140018220429E8D889
:10948000042CE6D805206043034A05331218525CC9
:10949000DDE7C046E865FF1FB0BE001110B50A0049
:1094A0001121024B00F0FBFA10BDC0466F9900116C
:1094B0000B0030B587B001AD2B806B460400110066
:1094C000981D082202F09CFA2A000B212000024B72
:1094D00000F0E5FA07B030BD9799001110B50A0009
:1094E0001121024B00F0DBFA10BDC046EB990011D0
:1094F00013B50B0011006A4613706B460400062278
:10950000581C02F07DFA6A4608212000014B00F049
:10951000C6FA13BD0B9A001110B50A001121024BB7
:1095200000F0BDFA10BDC0465B9A00117FB5050082
:109530000B4BAA00D4580800002C0FD0666F237F75
:10954000E28821780396266F0296E66E0196A46E55
:109550000094FDF709FC2800FFF7FAFD7FBDC04627
:10956000E865FF1F10B51721FFF7E0FF10BD0000F1
:1095700070B50A000D00064B0221040000F08FFABE
:10958000060029782000FFF7D1FF300070BDC046EB
:109590003B99001170B586B000236A46137083684A
:1095A00004001D78681E0A2859D801A902F000FBA2
:1095B000060633373B3F43474B4F5300180000F03C
:1095C00042F9062312284BD000281BD16088FFF7F0
:1095D000D9F90823002813D04279002A47D1264B15
:1095E0001A78072312070BD5244B1A680723002A81
:1095F00006D01668002E03D0290001AAB047030048
:109600006A4613706B461B786088002B2AD1FFF7DF
:1096100067FC06B070BD180000F06CF9D4E71800C4
:1096200000F087F9D0E7180000F093F9CCE71800B4
:1096300000F0ADF9C8E7180000F0C3F9C4E718005E
:1096400000F0F6F9C0E7180000F0F6F9BCE71800E2
:1096500000F013FAB8E7180000F013FAB4E7072394
:109660006A46137069466088FFF782FFD1E70523D9
:10967000012AC5D1024BB8E77564FF1FE065FF1FE3
:10968000E465FF1FF8B52C4F8600F35904000D0068
:10969000002B40D0DA8882423DD15A78062A33D155
:1096A0001A78002A2ED0012099681A6A097D014291
:1096B00006D0157B054203D007225A700120F8BD61
:1096C0000220014204D0157B054201D00922F4E7B3
:1096D0000420014204D0127B024201D00B22ECE7AD
:1096E000164B1B68002BE9D05B68002BE6D02000EE
:1096F0009847BB5900215B78122BDFD12000FFF780
:1097000015FFDBE70E4BECE7112A04D1002900D04E
:1097100032252900F2E7002D08D12000FFF732F9A9
:10972000002803D01023027913430371210028007D
:10973000FDF798FAC2E7C046E865FF1FE065FF1F26
:10974000E465FF1F70B50E4E8500AB590400002B79
:1097500013D01B78002B11D10A4B1B68002B04D0AF
:109760005B68002B01D02000984773595B78122B5F
:1097700003D100212000FFF7D9FE70BD024BECE7BA
:10978000E865FF1FE465FF1FE065FF1F094B8000D0
:10979000C3581020002B0CD01A6A002A09D09B68ED
:1097A000002B06D0127A1B7E101C9A4200D9181C7E
:1097B000C0B27047E865FF1F70B503000D001400CC
:1097C0000220002A30D000292ED013700B78081DFB
:1097D00053704B789370FFF7A7FCE07001200221D3
:1097E0002B7A23716B7B034063716A7B0A401343BE
:1097F000042263716E7B1640334363716E7BF608FF
:10980000F600334363712B7B0340A371287B014037
:1098100000200B43A371297B0A401343A3712A7BC9
:10982000D208D2001343A37170BD10B50A00010025
:109830000120FFF7C1FF10BD10B50A000100022092
:10984000FFF7BAFF10BD70B506000C000220002E15
:1098500030D000292ED07378201D0B70B3784B7058
:10986000F178FFF76DFC01223579257271794B1083
:1098700008001340934010400343881010408000BC
:10988000C9080343C9000B436373B1794B10080047
:109890001340934010400343881002409200C908CF
:1098A0001343C9000B4321202373FCF773FE854249
:1098B00001D2122070BD2220257AFCF76BFE854272
:1098C000F7D823781820042BF4D86378012BF1D82B
:1098D0000020EFE7030010B50220002909D0002B7B
:1098E00007D00322481C0A7019000D3202F088F8D4
:1098F000002010BD03000222080010B5002B06D086
:10990000002904D00E32591C02F07AF8002210000F
:1099100010BD030010B50220002909D0002B07D08C
:109920000422481C0A7019000C3202F069F8002069
:1099300010BD10B5FFF7DEFF10BD030002200029A7
:1099400006D0002B04D0052200200A701B784B7033
:10995000704703000220002B08D0002906D05B7856
:1099600000200B70013B082B00D918307047030012
:1099700010B50220002909D0002B07D00622481C70
:109980000A7019000A3202F03BF8002010BD10B531
:10999000FFF7B0FF10BD02000B00022010B5002938
:1099A0000ED0002A0CD00721197011885970118827
:1099B000090A997011180822D81C02F021F8002019
:1099C00010BD03000A00022010B5002B0CD00029A6
:1099D0000AD099785878090201431180901CD91C4B
:1099E000082202F00DF8002010BD030010B502207F
:1099F000002909D0002B07D00822481C0A70190042
:109A0000921801F0FDFF002010BD02000B000220A3
:109A100010B500290BD0002A09D00921197011783E
:109A200018185970511C062201F0EAFF002010BDE1
:109A300010B5FFF75FFF10BD02000B00022010B54C
:109A4000002A09D0002907D0517819701118062270
:109A5000581C01F0D5FF002010BD030010B50220F6
:109A6000002909D0002B07D00A22481C0A701900CF
:109A7000063201F0C5FF002010BD10B5FFF73AFF18
:109A800010BD02000B00022010B5002A06D00029EC
:109A900004D018005178FFF753FB002010BDF0B53B
:109AA00085B017001E006A46062305000800918154
:109AB0009380FEF7C0FC1324011E02900CD03800E6
:109AC000B047041E05D1280001A9FEF76FFA041E55
:109AD00002D0029801F034FE2800FFF701FA2000BE
:109AE00005B0F0BDF0B504008BB001911500002168
:109AF000102202A801F074FF334EA700B8590028C5
:109B00003CD0C388A34239D10378002B36D14278A8
:109B1000062A18D102000100553235310C3006AB4F
:109B2000FFF7A9FA002829D12000FFF72FFE020035
:109B300006A902A801F064FF200002A901F0F8FDC7
:109B400001200BB0F0BD816E002917D00B8A112ABD
:109B500028D19D420ED101981231093A01F0F0FF4F
:109B6000012807D1BB5920009D6EFFF70FFE290089
:109B70000200DEE732212000FFF7D8FC2000FEF7CC
:109B800001FF061E1BD0416A002918D00B8AAB4288
:109B900015D108220198123101F0D2FF01280ED10F
:109BA000716A0AE09D42E9D108220198123101F060
:109BB000C7FF0128E2D1BB59996E8A7EB9E7200020
:109BC00001F05EFDBCE7C046E865FF1FF0B56B4DD8
:109BD00087007E5985B0337802900393002B00D024
:109BE00087E0B368346A01937078062817D10122A0
:109BF0001B7D134202D0217B114218D10222134255
:109C000002D0217B114251D10422134203D0237B85
:109C1000134200D08BE0019B5A7DEB5991E007384D
:109C20000428F8D801F0C4FF032E42678300B36E06
:109C3000002B03D11C2001F04BFDB066EB599C6E4C
:109C4000002C1CD010220021200001F0C9FE029837
:109C5000FFF79CFD01002000FFF72DFA01F098FDB1
:109C60002082200008211230FFF725FA0298FFF722
:109C70008DFDA076EB592100D888FFF70FFC082254
:109C8000EB591CE0B36E002B05D01A00198AF0883E
:109C90001232FFF70DFC0222019B197DEB59114294
:109CA0003DD0207B10423AD0073208E0F488FCF720
:109CB000DBFD01002000FFF711FC0A22EB595A706E
:109CC000029B9C002A595378073B042B11D8D0885B
:109CD000FEF758FE00284ED0C3895A08D2182849EA
:109CE000029B0298CB542B5941180433254801F0AC
:109CF0009FFE05B0F0BDFCF79FFD030001208342ED
:109D000001D100200393EB59DE88FCF79BFD0399FA
:109D100002003000FFF7ECFB019AEB59117D0422A1
:109D200011420CD0217B114209D00B22C7E7F688E3
:109D3000FCF73CFD01003000FFF7EEFB6BE7019AFA
:109D4000527D01210A4204D0607B084201D00C22DE
:109D5000B5E702210A4204D0607B084201D00E22FE
:109D6000ADE704210A4204D0627B0A4201D01022EE
:109D7000A5E71222A3E7FA225200B0E7E865FF1F29
:109D8000EC65FF1F43A1001110B5064B1A780423A0
:109D9000100018401A4200D00348FFF727FA0020AD
:109DA00010BDC0467564FF1F2843FF1F70B5040037
:109DB000FFF7D4FA051E43D12000FFF77FFA234EA8
:109DC000A400A0598268937CDB0708D50321036AAD
:109DD0001B790B40012B02D1017F0B430377431DFD
:109DE000D97F8B1E022B0DD8022900D00121C088FB
:109DF000FCF790FF042133591A7F59700A431A77F0
:109E0000280070BD01290CD10223102243700021CB
:109E10000C3001F0E5FD305910213530FFF74BF9DA
:109E2000EEE70529ECD10223D118437010220C3043
:109E300001F0E6FD04233259117F0B431377EAE763
:109E400008251828DCD1053DDAE7C046E865FF1F84
:109E5000F0B58BB0059143887E4F9E00F4591500F4
:109E60000493002C15D1012902D000200BB0F0BDC5
:109E7000101D57781678FFF757F9EB6832000293F8
:109E80002B7A0499019300903B002000FCF70CFF13
:109E9000EBE7E388049A934201D00820E6E72378B1
:109EA000012B00D1D4E0059B581E092800D9CFE032
:109EB00001F07EFE05CE0A29CC506C859AB22900AD
:109EC0000498FFF773FFD1E72000290010224530E6
:109ED00001F096FDB9594B78042B02D1013B4B7030
:109EE000C3E70B000A00253335320C310498FFF725
:109EF00095F90498FFF702FA0522431E9841BB59D1
:109F0000C0005A70B2E7200029001022553001F03D
:109F100077FD049B4F4C9D00295904980A0006AB1D
:109F200055320C31FFF77AF929591022453106A82C
:109F300001F006FE012808D10498FFF7F7F9059013
:109F4000002804D106222B595A7005988EE7082361
:109F50000593FAE763780C2B7AD1E36E002B03D1DB
:109F60001C2001F0B5FBE066BB59D86E00286FD00D
:109F70001022290001F044FDBB590498DC6EFFF764
:109F800005FC0D22A076BB595A706EE7E06E0028E2
:109F90005ED063780D2B5BD12B8808220382A91C2D
:109FA000123001F02DFDBB599A68517D02221142F9
:109FB00026D0186A407B104222D00C32E4E7637846
:109FC0000E2B45D1236F002B03D1162001F080FB0F
:109FD0002067BB59186F002803D01022290001F018
:109FE0000FFD0F22BB59CFE763780F2B30D1206FC5
:109FF0000622691C103001F003FDBB599A68517D9F
:10A000000422114203D0196A497B1142D5D10021A3
:10A010000498FFF78BFA28E7636F002B0DD0BB592C
:10A02000586F0028F3D01022290001F0E9FC01222A
:10A03000BB5952425B6F1A61E9E7142001F048FBFB
:10A04000BB5960675B6F002BE9D126E72978DFE712
:10A0500007200BE7E865FF1F10B5064C207001F0E4
:10A060008FFD06212078FDF791FF0348FEF778FC6D
:10A0700010BDC046FB65FF1FF991001100200BB217
:10A0800070B50D00834216DA264B187801F0C0FB3C
:10A09000041E0DD00378922B0ED0A02B37D0224B6C
:10A0A0001878FF283AD0210001F082FC002835D131
:10A0B00080200002684070BD43780E2B0BD03E2BF1
:10A0C000EDD18378052B12D0082BE8D181798088D7
:10A0D000FFF7D8FA08E0154B82889A42DFD18368EF
:10A0E0001878591CFEF7C0FE002817D1D7E7104B8F
:10A0F0001B785B0712D50F4B1B68002B0ED09B689B
:10A10000002B0BD0C289811D80889847ECE7FFF7B0
:10A1100041FAA068002801D001F012FB200001F0F4
:10A12000B7FAC5E7FB65FF1F2143FF1F182000009A
:10A130007564FF1FE465FF1F10B50078FFF712FA82
:10A1400010BD10B50078FFF7FDFA10BD0C23434396
:10A15000084A10B59B185A68002A03D0012901D17A
:10A16000904710BD9B68002BFBD00029F9D1984780
:10A17000F7E7C0461866FF1F01238340094A10B560
:10A18000946B1C439463506B98435063D46B2000D2
:10A190009843012901D120001843D063116B0B4370
:10A1A000136310BD00800040F0B500240127154B5B
:10A1B00085B0DA6B144E03921A6C0192DA64019B3B
:10A1C000E3403B4217D0039DE5403D400295E5B298
:10A1D00002992800FFF7BAFF316A736A002908D094
:10A1E0003900002B01D0029979402800FFF7C4FF05
:10A1F00001E0002BF9D101340C36172CDFD105B06A
:10A20000F0BDC04600800040FC65FF1F064B0121E9
:10A210005A68C2400A4204D01B68C3401800084074
:10A2200070471B6DF9E7C046008000400122064BD5
:10A230008240002903D0D9680A43DA607047D968A0
:10A240009143D960FAE7C0460038004030B5032496
:10A2500044430F4BE25C1B199C785D7801232D1B56
:10A260000135AB40013BA340A140DB430C00122869
:10A2700007D808499200521811681940214311600B
:10A2800030BD054A11680B4023431360F8E7C04610
:10A29000F7BE001108F0004014F00040C21F70B576
:10A2A000D4B20623092C0BD80125084C954000296F
:10A2B00008D00021FFF7CAFF23682B432360002347
:10A2C000180070BD2368AB43F8E7C0460038004073
:10A2D000214BF0B51B185B78022B21D1032444439A
:10A2E0001E4A1F4EA35C1219947801221500854066
:10A2F000B76B013CE4B23D43A240B563194C122850
:10A3000015D89B0000290CD117495B1899680A439E
:10A310009A600123205C154A834011680B43136047
:10A32000F0BD11495B18996891439960F1E70E4BB4
:10A3300000290DD159690A435A61225C1328E8D0DB
:10A340000123203A93400A49086803430B60E7E77A
:10A35000596991435961F0E7FC65FF1FF7BE001191
:10A36000008000403CBF001100F00040A0F0004021
:10A37000A4F00040F8B500241B4E1C4D1C4B1B5D87
:10A38000012B1FD1194A9269E2401A420BD00122D7
:10A39000B25693402200143AD2B2022A09D8154983
:10A3A0004A6913434B61013402360C35172CE5D151
:10A3B000F8BD0022B2560F499200521891680B4323
:10A3C0009360F0E7022BEED1E7B23800FFF71EFFF3
:10A3D00001235840C1B23800FFF77AFF3800FFF779
:10A3E00015FF6877DFE7C046C9BE0011FC65FF1F97
:10A3F000FD65FF1F00F00040012202388240054B3E
:10A40000002903D059690A435A6170475969914339
:10A410005961FAE700380040F8B50E0001210F003D
:10A420008740114A0400D368FD43BB43D360831EB9
:10A430008B4201D8FFF7E0FF00212000FFF72EFF3D
:10A440000A4A0B4B5168012E05D139431B19516043
:10A450005E700020F8BD2940516002221C19627014
:10A460009A6915409D61F4E7003800400080004083
:10A47000FC65FF1F012210B58240074B002906D062
:10A4800019680A431A600121FFF7C6FF10BD196859
:10A4900091431960F7E7C046008000400C2370B577
:10A4A000002543430A4A29009B181D70094B0400EC
:10A4B0001B185D70FFF7B0FF0123A3400649280079
:10A4C0000A681A430A6005490A689A430A6070BD1F
:10A4D0001866FF1FFC65FF1F34800040308000407D
:10A4E00070B504000E00FF2813D003250540FFF7C8
:10A4F000D5FF084AA3089B009B183F22ED00AA4005
:10A50000AE40196820009143314319600121FFF7E3
:10A510008DFE70BD18380040F8B50C244443134B31
:10A520000500E4186368002B03D1A3681220002BF8
:10A530001AD0022201270E4B00215B195A70280005
:10A540002770FFF769FF63681E1E08D0A3683E00EE
:10A55000002B04D02800FFF759FE4640F6B2280031
:10A560003100FFF709FE0020F8BDC0461866FF1F46
:10A57000FC65FF1FF7B5C420FF222B4B8000195844
:10A58000002491433F3A0A431A508022274F520237
:10A59000274E1A60274B1D5D002D21D0A31E012BD5
:10A5A00003D80121E0B2FFF727FF012D18D11F4B7F
:10A5B0009B69E3402B4213D0E3B218000193FFF7ED
:10A5C00025FE01000198FFF755FFE3B2143B022B73
:10A5D0001DD801217156184A8D405369AB43536110
:10A5E0003B7F002B0DD0E5B22800FFF795FF280038
:10A5F000FFF70CFE7B7F0100834202D02800FFF7AB
:10A60000A5FD01340C370236172CC3D1F7BD01214B
:10A6100000237156F3568D40074A9B009B189A6899
:10A62000AA439A60DCE7C04600E100E0FC65FF1F3A
:10A63000C9BE0011FD65FF1F00F0004010B50121EB
:10A640000400FFF7E9FE0123044A002011194B70B2
:10A65000A34091690B43936110BDC046FC65FF1F89
:10A6600070B50E0015000400FFF718FF0C236343BC
:10A67000094A20009B189D605E60FFF74DFFF021A6
:10A68000064B074A8900051E5A5002D02000FFF7EA
:10A6900005FF280070BDC0461866FF1F0000FF1FA1
:10A6A000A9A1001170B5134D07202C78002C1FD1E3
:10A6B000982221005200280001F09AFA0123C420B8
:10A6C000FF222B700C4B80001C635C630B4B1C60E7
:10A6D0005C600B4B195891433F3A0A431A50802251
:10A6E00052021A600D20074A074900F0A1FF20001E
:10A6F00070BDC046FC65FF1F00800040A0F0004018
:10A7000000E100E075A5001175A30011030010B56C
:10A710000620072B09D8054A137001F079FAD721D2
:10A720000020034B034A89005A5010BD5043FF1FBD
:10A730000000FF1F8D1BFF1F70B51D0002240C2998
:10A7400010D8094ACA40D2070CD5FBF72FFF041EC8
:10A7500008D1059A04992800FBF744FFFCF7B2FDE5
:10A76000FFF712FB200070BD1210000030B50D780D
:10A7700002232C009C43184201D02B431C000825C7
:10A780002300AB43284201D02B00234320241D008B
:10A79000A543204201D01C4325002A230D701842F6
:10A7A00004D011781E3B0B43137030BD0028FCD140
:10A7B0000C2113788B43F7E7F8B51D0006AB1B8817
:10A7C000140007AA0E000B201778002B27D10A7857
:10A7D000022A49D14A68507811780002244A084375
:10A7E0008018042840D801F0E3F903121D1B230050
:10A7F000F06800F05DFF021CC0B2B84200D93A1CFC
:10A80000D2B22000F1682A8001F0FAF806E00222B4
:10A81000F3681B882A8023701B0A63700020F8BD30
:10A820000622EEE701232B80F3681B782370F5E7FF
:10A83000F368002B16D008222A801A8822701A8802
:10A84000120A62705A88A2705A88120AE2709A88B4
:10A8500022719A88120A6271DA88A271DB881B0A57
:10A86000E371DBE72B80D9E701202B80D7E7C046D7
:10A8700000D6FFFFF7B516000A781D0008AB1F8849
:10A880000C000123022A18D14A685078117800027E
:10A890002B4A0843801803280FD801F089F90225B4
:10A8A0004439E06800F004FFC0B20723B84204D383
:10A8B0007B190193152B02DD0D231800FEBDE06806
:10A8C0002A003100C01901F09BF86B4600209B88DC
:10A8D000E268D0541B4B1B68834203D01B68834241
:10A8E00000D098470023E8E70B23002FE5D1022D85
:10A8F000E2D1737832781B021343E2681380114B64
:10A900001B68002BEED01B68002BEBD00120E8E782
:10A910000B23002FD1D1062DCED12A003100E068C3
:10A9200001F06EF8DEE70B23002FC6D1012DC3D155
:10A9300032787533012AC0D8E3681A70D2E7C0466E
:10A9400000D6FFFF0868FF1F70B50C001500072830
:10A9500037D801F02DF9041436361B36242E182072
:10A9600015290BD8184E16220021300001F038F8B6
:10A9700022002900300001F043F8002070BD1820AB
:10A980000229FBD11288114B1A80F6E718200829FA
:10A99000F4D10A000E48290000F01AFFEDE7182054
:10A9A0000129EBD10B4B10780B49DA69FFF7DEFE7A
:10A9B000E3E718200129E1D1064B10780749DA6B4B
:10A9C000F4E70220DAE7C046F067FF1FCE43FF1F1F
:10A9D000C443FF1F5443FF1F7C43FF1F9C43FF1FC3
:10A9E000030010B50020DB0704D50721024A034805
:10A9F00000F08CF810BDC04654BF00115443FF1F37
:10AA0000054A03001068002803D082889A4201D1C9
:10AA1000806870470068F6E7006AFF1F0A88030035
:10AA200008009A4204D08A8804309A4200D000205C
:10AA300070470000F8B5F22200230D4F0D4E7968E3
:10AA4000050042433370994200D07B600A4C0021DC
:10AA5000200000F0C5FF00231A007C60AB4202D149
:10AA600000203370F8BD01332280DBB2F234F5E709
:10AA7000F86AFF1FF66AFF1F046AFF1F73B56B4673
:10AA800001900600684615001980FCF74DFF041E72
:10AA900011D1002D0FD07689002E11D00C2000F09E
:10AAA00017FE00280ED0084A04601368868085606F
:10AAB000002B02D11060200076BD1A001B68F7E75A
:10AAC0000224F8E71324F6E7006AFF1F01210022A1
:10AAD0000A4B10B549420A4C198099809A719A70B4
:10AAE000084B2070012019805A60FFF7A3FF2078DF
:10AAF000FCF778FF0448FDF733FF10BD1068FF1F17
:10AB0000006BFF1FF86AFF1FB9AB0011022310B5DD
:10AB1000002802D0FFF7B2FF0300180010BD0000AC
:10AB2000030010B50020DB0704D50421024A0348C6
:10AB3000FFF7A4FF10BDC04668BF0011D443FF1F3C
:10AB4000F0B50E2687B003930CAB1F8802ABF61846
:10AB50000500080031000292FDF768F804000120AA
:10AB6000002C0FD03088FFF74BFF03000E20002B86
:10AB700008D05E68002E05D021002800039B029AB1
:10AB80000097B04707B0F0BD0A4B10B5984207D107
:10AB90000122002352420A808B708A808B7110BD83
:10ABA000FFF73CFF0028FAD001235B42038000231B
:10ABB0008370F4E7FFFF0000F8B5050001290AD112
:10ABC000134E00243388F227AB4219D028001149D4
:10ABD000FFF7DAFF06E0022904D10139FDF73EFF55
:10ABE0000028EDD0F8BD3B0063437268D018D35AFB
:10ABF000002B09D03A00002100F0F2FE0134E4B24B
:10AC0000054B1B78A342EED801235B423380DDE77E
:10AC1000F86AFF1F1068FF1FF66AFF1F10B5FFF7E5
:10AC2000FDFE03000020834200D0987810BD000094
:10AC3000F0B589B01C000EAB80CB03901E8810AB22
:10AC40001B78049202930B7A0D00DB0616D42B7846
:10AC50000593022B24D00498FFF7D2FE002812D0CF
:10AC600003689C46002B0ED0029B22000193290012
:10AC70003B00644603980096A04705E00498FFF760
:10AC8000BFFE002802D10E2009B0F0BD8368002B62
:10AC9000F9D00A222900039898470028D7D0F3E773
:10ACA0006B6858781A786B4B000210439842D2D8E0
:10ACB000043B984210D2684B984242D015D8674B5B
:10ACC000C0180128C7D80B20002EDDD1EB681A78F8
:10ACD00059683A80200028E0614BC018032800D949
:10ACE00079E000F065FF846A789E5E4B9842B2D1AD
:10ACF0000B20002EC8D101233B80EB6831001B786C
:10AD000023706889013080B2FCF790FF3A88031EF7
:10AD10000ED0017802328A183A80428962704289E4
:10AD2000120AA27059680278E01C00F069FE06E081
:10AD300004323A8031000422601C00F051FE0020F1
:10AD4000A2E70B20002E9FD1EB6807A91E880423E1
:10AD50003B80330A300026706370FCF767FF051EE6
:10AD600028D004AB9A890E2304A95B183E49C66813
:10AD7000FCF7D0FF00280BD12B783C486A68059976
:10AD8000FBF786FB002803D1012304AA5B42D38191
:10AD90003278022A06D17168201D00F031FE3B880E
:10ADA00002333B800E2304AA9B181B88A3701B0A46
:10ADB000E370C4E704ABDE81F4E70B20002E00D083
:10ADC00062E7E9680398FFF729FF02233B802070C0
:10ADD000000A6070B3E70B20002E00D054E7022277
:10ADE000EB681B883A8023701B0A6370A7E7E8684A
:10ADF00000F05EFCC2B203000720B24200D243E77B
:10AE00000DD00299DBB27118994202DB921BD3B2CA
:10AE10000293029BE9681A003B8089195AE70023D4
:10AE2000F6E70B20002E00D02EE70722EB683A80D1
:10AE30001A7822705A7862705A88A2705A88120A58
:10AE4000E2701A792271DA886271DB881B0AA371B9
:10AE500075E7C046042900000228000000D8FFFF63
:10AE6000FFD6FFFF03280000FFFF000098BE00117F
:10AE7000F0B58DB06B460020089120229B5E834286
:10AE80003DDAA64B187800F0C3FC071E32D00378D9
:10AE9000B02B2CD10079023816281FD800F0E0FD25
:10AEA00017001E001E001E0031001E0096001E002E
:10AEB0001D011E0052011E0073011E00CD011E0067
:10AEC00050021E001E001E008E021E00E302944B64
:10AED00094491B8878880B80FBF71AF83800FCF738
:10AEE0009BFF914B1B68002B01D03800984738001E
:10AEF00000F0CEFB8020089B0002434018000DB0FC
:10AF0000F0BDEE220021874800F06AFD0BAA3B7BD2
:10AF10007989388900923A000D32FCF79FFD0400D0
:10AF2000804B1B78002C3FD146E0804B78880593FE
:10AF30007F4B4100CB5A0BAE073BDBB2328802930A
:10AF4000002301937B4B210006930093059BFFF7A1
:10AF50006FFE744D002810D1069B3A8A1B889A42D6
:10AF60000BD138000599123000F0EAFD002804D01A
:10AF70002B7862899B00EB185A80162306A81B18B1
:10AF8000328820007989FCF7C5FE2B7804009A00EE
:10AF9000AA1851880029C3D00133DBB22B700028D6
:10AFA00007D006A9C98A9180634A12889A42BCD800
:10AFB00002E0012149429180002B04D05949788850
:10AFC000FAF7DAFF8AE73E890A2479E000253E890C
:10AFD000574B06937B88069A5B009B5A033B9D4226
:10AFE00002DB002DF0D05BE0162206A812183B7B96
:10AFF000798900923A0030000D32FCF72FFD059060
:10B00000002858D04689017A7888FCF7F1FC041EA4
:10B0100044D1464B78880793069B4100C95A454B5B
:10B020000439C9B206AAD28A069302910194009308
:10B030000599079BFFF7FCFD041E2FD1069B39499C
:10B040001A88931C002D26D14B807988384B4900F3
:10B05000CB5A5119033B8B4220DD059B31485B895C
:10B0600041190B71A91C0135C9B2EDB20591451901
:10B070001B0A2B71059B2D490433181800F0C0FCE6
:10B080002C4B059A1B88D318DDB22C4B9E4205D061
:10B090000136B6B29CE749889942D6D0002D0CD033
:10B0A000204C2800618800F06BFC2070210078881B
:10B0B000FAF772FF12E7059CF0E7002C00D183E756
:10B0C0007B78142B00D109E716493B794E800B7031
:10B0D0000C717888FAF712FF00E7162406ABE41823
:10B0E00021003889FCF7A2FD011E00D1B7E1788864
:10B0F00022880F4C45002C5B0A4D013CE4B20294BF
:10B1000000240F4B01940095FFF792FD041E00D020
:10B1100014E129007888FAF74FFFDFE6006BFF1F84
:10B12000C042FF1F1868FF1F0C68FF1F0C69FF1F3C
:10B130004864FF1FFC69FF1FBE42FF1FFFFF0000A6
:10B140001A68FF1F162406ABE41821003889FCF7A3
:10B150006DFD011E00D182E178882288AE4C450049
:10B160002C5BAE4D013CE4B202947C89AC4B019463
:10B170000095FFF75DFD041E00D0DFE02900788810
:10B18000FAF724FFAAE60025A44B1D803B00F63306
:10B190001B78A24A78880792AB4208D99E4B128846
:10B1A0000693069943005B5A013B9A4203DB0799D9
:10B1B000FAF716FF92E616246B00FB18059306AB10
:10B1C000E418059B21001889FCF730FD011E03D10E
:10B1D000059B01241E8973E77888924B2288069C80
:10B1E000099343001B5B904E013BDBB202930023AB
:10B1F00000960193099BFFF71BFD041E02D0059BDF
:10B200001E895DE77B88069A5B009B5A079A108827
:10B2100032881218934202DC1B1A013B33807F4CA8
:10B22000023032880999001900F0EAFB238832883D
:10B2300001359B182380EDB2A8E70BAA3B7B7989E7
:10B24000388900923A000D32FCF708FC0025059081
:10B25000059B002B04D10A24002D00D16EE060E094
:10B26000059B7888197AFCF7C3FB0100041E63D1A3
:10B27000694C6C4B788806940993069B4400E45A09
:10B28000694B063CE4B20BAE3288079302940191FD
:10B2900000930599099BFFF7CBFC041E4CD1079B3B
:10B2A0005E491B881A1D002D30D14A80059B5B4CDE
:10B2B0005A8963191A716B1C9BB2E318120A1A712E
:10B2C000162306A832881B1879890598FCF722FDF9
:10B2D000FF21AA1C2E1D03350B00059092B2B6B2B9
:10B2E000ADB2002803D006ABDB8AD9B21B0AA21884
:10B2F000651911712B714C4D301D2A884949201850
:10B3000000F07EFB2B88F618B5B2A1E74988914280
:10B3100007D17A8806995200525AEB18053A9A4298
:10B32000C4DC3E4C2800618800F03AFA207021000D
:10B330007888FAF75FFED1E5002DF2D13E89BFE6AD
:10B34000162606ABF61831003889FCF76FFC3D0075
:10B350000400FA3500282DD0037A9B060CD4002275
:10B360007B893989788800923A000C32FFF7E8FB34
:10B37000041E10D03E8915E03088FFF741FB0028FD
:10B380001AD08368002B17D02100122278889847A2
:10B39000041EE4D0EEE72B78002B02D17888FAF770
:10B3A00039FE00262B78002B00D097E5002C00D129
:10B3B00094E585E60124DDE70E24DBE7162506ABE0
:10B3C000ED1829003889FCF731FC041E47D0037AB8
:10B3D0009B0611D4154A7B881188994203D01448E2
:10B3E000814207D11380134BF2261D780023D9B276
:10B3F000A94221D30924A1E72888FFF701FB0028EF
:10B400002FD08368002B2CD02100122278889847F7
:10B41000041EDFD092E7C0464864FF1F1868FF1F74
:10B420001A68FF1F0C69FF1FFC69FF1FF86AFF1FE6
:10B43000FFFF0000F66AFF1F3100594354680133D3
:10B440006018615A0029D2D13C0008342100F22250
:10B4500000F0D6FA21007888FAF7E4FD3EE50124F1
:10B460006CE70E246AE71D4B1A887B889A4231D01C
:10B470007888FAF7E1FD31E5F223059851684343F6
:10B48000CD18C95A00291FD03B7A012B0BD16C88EB
:10B49000AB887888AA1D0094FFF752FB041E02D0E7
:10B4A00000233B722E88F2220021280000F098FA37
:10B4B00000232B80059B0133DBB20593084B0599D4
:10B4C0001B78064A8B42D7D801235B421380002C9D
:10B4D000CED0F5E5002634000596EFE7F86AFF1FA9
:10B4E000F66AFF1F70B504000E001500FFF796FA0C
:10B4F000031E08D131000548FFF790FA0300112020
:10B50000002B02D01C8000209D7070BDFFFF00004A
:10B51000F8B50B4F06003B780D001400FF2B0ED042
:10B520000A2000F02DF9011E09D0B1230380002369
:10B5300046800371C5800481387800F039FAF8BD7F
:10B540001544FF1FF7B50F0008A90600088809A9D0
:10B550000B240988002821D10234022B1ED15578F2
:10B5600013782D021D432B008B4301937334002B62
:10B5700014D1FB68300019000093FFF74FFB019CCA
:10B5800085420BD02A0030000099FFF7ABFF041E64
:10B5900004D12A0030007989FFF7BAFF2000FEBDF0
:10B5A000F0B50E7885B003900AA805880120022E18
:10B5B0000DD14C682778647824023C43054FBC4287
:10B5C00005D10398DBB201960095FFF7BBFF05B0EC
:10B5D000F0BDC04602290000034B10B51B68002BCC
:10B5E00000D09847FEE7C046046BFF1F07B501A8CF
:10B5F000FFF7F2FF044A05480021121A00F0F8FA9A
:10B60000F8F7F8F8FEE7C046086BFF1F1844FF1F65
:10B6100001B40248844601BC604700BFC9A90000CC
:10B6200001B40248844601BC604700BF55220000B7
:10B6300001B40248844601BC604700BF0D31FF1FC2
:10B6400001B40248844601BC604700BF156B01008D
:10B6500001B40248844601BC604700BFF938FF1FAF
:10B6600001B40248844601BC604700BFA54F0100F9
:10B6700001B40248844601BC604700BF8D1200003F
:10B6800001B40248844601BC604700BF091B0000AA
:10B6900001B40248844601BC604700BF434D01002D
:10B6A00001B40248844601BC604700BFE548000081
:10B6B00001B40248844601BC604700BFDD5201006E
:10B6C00001B40248844601BC604700BF014C010040
:10B6D00001B40248844601BC604700BF3D4B0100F5
:10B6E00001B40248844601BC604700BF2124000029
:10B6F00001B40248844601BC604700BFED4A010026
:10B7000001B40248844601BC604700BF8552010075
:10B7100001B40248844601BC604700BF993AFF1F4C
:10B7200001B40248844601BC604700BF8B5201004F
:10B7300001B40248844601BC604700BF311B0000D1
:10B7400001B40248844601BC604700BFD9490100EA
:10B7500001B40248844601BC604700BF456B01004C
:10B7600001B40248844601BC604700BF056A00007E
:10B7700001B40248844601BC604700BF3139FF1F55
:10B7800001B40248844601BC604700BF1D4D010062
:10B7900001B40248844601BC604700BF2951010042
:10B7A00001B40248844601BC604700BF090E000096
:10B7B00001B40248844601BC604700BFC94A010089
:10B7C00001B40248844601BC604700BF055E00002A
:10B7D00001B40248844601BC604700BF810E0000EE
:10B7E00001B40248844601BC604700BF55490100CE
:10B7F00001B40248844601BC604700BF7139FF1F95
:10B8000001B40248844601BC604700BF51250000D6
:10B8100001B40248844601BC604700BFF54E0100F8
:10B8200001B40248844601BC604700BFF30E00002B
:10B8300001B40248844601BC604700BF0534FF1FC5
:10B8400001B40248844601BC604700BF291C0000C7
:10B8500001B40248844601BC604700BF090E0000E5
:10B8600001B40248844601BC604700BF75A90000CE
:10B8700001B40248844601BC604700BFB3520100D6
:10B8800001B40248844601BC604700BFE538FF1F91
:10B8900001B40248844601BC604700BF1147010063
:10B8A00001B40248844601BC604700BFF94C010066
:10B8B00001B40248844601BC604700BF6DBC000073
:10B8C00001B40248844601BC604700BF45500000F7
:10B8D00001B40248844601BC604700BF3D18000027
:10B8E00001B40248844601BC604700BF3D37FF1FDA
:10B8F00001B40248844601BC604700BFADAE000001
:10B9000001B40248844601BC604700BFF137FF1F05
:10B9100001B40248844601BC604700BF3119FF1FD3
:10B9200001B40248844601BC604700BF4D1F0000BF
:10B9300001B40248844601BC604700BFE117000023
:10B9400001B40248844601BC604700BF8530FF1F38
:10B9500001B40248844601BC604700BF6D36FF1F3A
:10B9600001B40248844601BC604700BF9DA90000A5
:10B9700001B40248844601BC604700BF0519FF1F9F
:10B9800001B40248844601BC604700BF350E000088
:10B9900001B40248844601BC604700BF350E000078
:10B9A00001B40248844601BC604700BFB54C0100A9
:10B9B00001B40248844601BC604700BF594F0100F2
:10B9C00001B40248844601BC604700BF5D17000017
:10B9D00001B40248844601BC604700BF2146010013
:10B9E00001B40248844601BC604700BF154D010008
:10B9F00001B40248844601BC604700BF1D3AFF1FE6
:10BA000001B40248844601BC604700BFE94C010014
:10BA100001B40248844601BC604700BF6D30FF1F7F
:10BA200001B40248844601BC604700BF691F0000A2
:10BA300001B40248844601BC604700BFA94601002A
:10BA400001B40248844601BC604700BF2D2EFF1F91
:10BA500001B40248844601BC604700BFC51D000018
:10BA600001B40248844601BC604700BF313BFF1F60
:10BA700001B40248844601BC604700BF5147010041
:10BA800001B40248844601BC604700BF0D5201006A
:10BA900001B40248844601BC604700BFED3AFF1F75
:10BAA00001B40248844601BC604700BF3D36FF1F19
:10BAB00001B40248844601BC604700BF65710100C3
:10BAC00001B40248844601BC604700BF45510100F3
:10BAD00001B40248844601BC604700BFAD32FF1F7D
:10BAE00001B40248844601BC604700BF093BFF1F08
:10BAF00001B40248844601BC604700BFE928000049
:10BB000001B40248844601BC604700BF25260000FE
:10BB100001B40248844601BC604700BF4936FF1F9C
:10BB200001B40248844601BC604700BF595201007D
:10BB300001B40248844601BC604700BFC56D0100E6
:10BB400001B40248844601BC604700BFCD4C0100EF
:10BB500001B40248844601BC604700BFEDA5000067
:10BB600001B40248844601BC604700BFB139FF1FE1
:10BB700001B40248844601BC604700BFD91B0000E5
:10BB800001B40248844601BC604700BFC9260000DA
:10BB900001B40248844601BC604700BF7918000028
:10BBA00001B40248844601BC604700BFB14E0000AA
:10BBB00001B40248844601BC604700BF1D3BFF1F23
:10BBC00001B40248844601BC604700BF851F0000E5
:10BBD00001B40248844601BC604700BFC521000093
:10BBE00001B40248844601BC604700BF0124000044
:10BBF00001B40248844601BC604700BFB70E000094
:10BC000001B40248844601BC604700BFD532FF1F23
:10BC100001B40248844601BC604700BF8D1BFF1F72
:10BC200001B40248844601BC604700BF017F0000A8
:10BC300001B40248844601BC604700BFC53AFF1FFB
:10BC400001B40248844601BC604700BFDD660100C4
:10BC500001B40248844601BC604700BF355500006E
:10BC600001B40248844601BC604700BF1D4B01007F
:10BC70000001010302000303040305020602070298
:10BC8000080209020A030B030C020D000E030F0346
:10BC9000100311001300140315001600AD3B001132
:10BCA000E13B00110000000002000000B2BC0011E6
:10BCB000192A0F180A000000F1590000FD240000A5
:10BCC00041460100698000117DA00011D17400116E
:10BCD0006D7E00113553001171AE0011814F0011BE
:10BCE000BD3D0011ED3E00110000000016160000E1
:10BCF00002000000FCBC0011F4FFF3FFD2FC0000C6
:10BD00002D40001100000000000000005475796112
:10BD10000042312E34003030313900676974687563
:10BD2000622E636F6D2F70767678005448303546FA
:10BD3000000000000200000048BD0011292A282A46
:10BD4000272A262A252A242A0A180000E2040000AD
:10BD50007102000078EC0000744000001027000021
:10BD600060F0000006640000204E000000000000AB
:10BD7000050000001F501D00023CB4000001190026
:10BD800014000000A1020000303132333435363760
:10BD900038394142434445460000000039570011FC
:10BDA0008D5700110000000002000000B4BD00111A
:10BDB0006F2A6E2A1A18EAD8BC80F0FC60000000D6
:10BDC00000000000000000F505D39727B6F615F730
:10BDD000B777E6F0C7F27200000001A00000000093
:10BDE0006410B71DC8206E3BAC30D9269041DC767C
:10BDF000F4516B6B5861B24D3C7105502083B8ED26
:10BE000044930FF0E8A3D6D68CB361CBB0C2649B49
:10BE1000D4D2D38678E20AA01CF2BDBDFB349B5F6E
:10BE2000800000800010000000000000D3600011BE
:10BE30005D770011F7600011657B00117B610011D7
:10BE40003B7B0011F1610011117B00114362001175
:10BE5000D97C0011AB620011D97C0011DD620011A8
:10BE6000937C0011F1610011C97A0011696200111F
:10BE7000717C001100000000000000004F63001101
:10BE8000717C0011B163001175770011052A042A35
:10BE9000012A002A02290328012800280118001875
:10BEA000000000000000000000000000000000870B
:10BEB0000101020102010102010203030401030165
:10BEC000010101010303020103000D000E00100037
:10BED000110013001401070108010A010B011C01E4
:10BEE0001D02040205020702080219021A021C02BE
:10BEF0001D030103020317000201000504000807E7
:10BF0000000B0A001716001D1C01020101050401A7
:10BF10000E0D011110011413011716011A19020256
:10BF200001020B0A020E0D02111002141302171661
:10BF3000030504030807030B0A030E0D00010203A7
:10BF400007090A0B0E0F101112141718191A1B1FCC
:10BF500020212200B9A7001175A8001100000000DF
:10BF6000020000009EBE001100000000A1B50011FB
:0CBF700000000000020000009CBE001158
:020000041FFFDC
:1000000000000000253D0011B8BC0011B4BC001177
:100010004861FF1F00000000000000000000000019
:1000200000000000000000000000000000000000D0
:1000300000000000000000000000000000000000C0
:1000400000000000000000000000000000000000B0
:1000500000000000000000000000000000000000A0
:100060000000000000000000000000000000000090
:100070000000000000000000000000000000000080
:100080000000000000000000000000000000000070
:100090000000000000000000000000000000000060
:1000A0000000000000000000000000000000000050
:1000B0000000000000000000000000000000000040
:1000C0000000000000000000000000000000000030
:1000D0000000000000000000000000000000000020
:1000E0000000000000000000000000000000000010
:1000F0000000000000000000000000000000000000
:1001000000000000000000000000000000000000EF
:1001100000000000000000000000000000000000DF
:1001200000000000000000000000000000000000CF
:1001300000000000000000000000000000000000BF
:1001400000000000000000000000000000000000AF
:10015000000000000000000000000000000000009F
:10016000000000000000000000000000000000008F
:10017000000000000000000000000000000000007F
:10018000000000000000000000000000000000006F
:10019000F932FF1F5931FF1FC16601000000000046
:1001A000000000000000000000000000000000004F
:1001B000000000000000000000000000000000003F
:1001C000000000000000000000000000000000002F
:1001D000000000000000000000000000000000001F
:1001E000000000000000000000000000000000000F
:1001F00000000000000000000000000000000000FF
:1002000000000000000000000000000000000000EE
:1002100000000000000000000000000000000000DE
:1002200000000000000000000000000000000000CE
:1002300000000000000000000000000000000000BE
:1002400000000000000000000000000000000000AE
:10025000000000000000000000000000000000009E
:10026000000000000000000000000000000000008E
:10027000000000000000000000000000000000007E
:10028000000000000000000000000000000000006E
:10029000000000000000000000000000000000005E
:1002A000000000000000000000000000000000004E
:1002B000000000000000000000000000000000003E
:1002C000000000000000000000000000000000002E
:1002D000000000000000000000000000000000001E
:1002E000000000000000000000000000000000000E
:1002F00000000000000000000000000000000000FE
:1003000000000000000000000000000000000000ED
:1003100000000000000000000000000000000000DD
:1003200000000000000000000000000000000000CD
:1003300000000000000000000000000000000000BD
:1003400000000000000000000000000000000000AD
:10035000000000000000000000000000000000009D
:10036000000000000000000000000000000000008D
:10037000EDB50011000000000000000000000000CA
:10038000000000000000000000000000000000006D
:10039000000000000000000000000000000000005D
:1003A0000000000000000000000000000D1BFF1F07
:1003B000000000000000000000000000000000003D
:1003C000000000000000000000000000000000002D
:1003D000000000000000000000000000000000001D
:1003E000000000000000000000000000000000000D
:1003F00000000000000000000000000000000000FD
:08183800106FFF1F4118FF1F94
:10184000024981F3088802F0F7FA0000106FFF1FC9
:1018500070B500241E491F4A1F484C6308CA1B0567
:101860001B0DE4188242F9D11C4B80228B630021AE
:1018700009201B4B920519621A4B1B4DDA671B4B53
:10188000DA688243DA609A68194802409A60112047
:10189000296002F08DF8112002F06AF880226B6C4A
:1018A000112093436B64EE23DB006343114A1B0C4E
:1018B00013840122104B9A7201F004FC0F4B1B7829
:1018C000002B04D10E4B1021187802F025FA70BDC0
:1018D000000005408805054000060540FF010000A6
:1018E00000F0004004E100E0003800403CF000401F
:1018F000FFDFFFFF1861FF1FCC61FF1FFA63FF1FAF
:10190000F861FF1F10B502F027F9072804D012284C
:1019100008D0022808D010BD044A0420136B0133FC
:101920001363F8E70220F6E71420F4E7F064FF1FE2
:10193000F8B507000C0026002500503630785135E8
:10194000002804D10300287058342370F8BD29788A
:10195000CA00481E8141A3183800A25C5B68C9B266
:10196000FFF7D0FF00280DD12B78DA00A218013341
:1019700050602B703378044A013B3370136A013393
:101980001362D8E70123DFE7F064FF1F5C234343C2
:10199000074910B5C9180B0058331B78012B05D126
:1019A000FFF7C6FF034A936A0133936210BDC04636
:1019B0002465FF1FF064FF1F10B502F035FB064AD7
:1019C0000121130010CB4942D967044B136002F088
:1019D0004BF9200010BDC04600E100E010001000EF
:1019E00010B5040002F020FB024B1C6002F03CF931
:1019F00010BDC04600E100E0431E5A425341A02200
:101A0000F0B5D2015B421340154D164A40019B18B8
:101A10002A18127E8BB00191002A1BD01A000832BE
:101A2000D46F0022E6B206AFE4B294420EDC28186E
:101A3000C369002B08D0019902AA117106AA049269
:101A400002AA167303A898470BB0F0BD1978B954D1
:101A50000132EAE71A7D1A7806AB01261A70E6E72A
:101A6000B067FF1F00400040F0B5254B0400400167
:101A7000C25C85B0002A2BD01A18117E002927D00D
:101A8000917E002924D01179022921D11689D78885
:101A9000D168F51BADB22A1C102D00D9102292B2CC
:101AA000BE4217D11818012303710023C269C380F5
:101AB00003819A4206D068460321037301710293A1
:101AC00001A890470820002C00D0192001F0FAFA54
:101AD00005B0F0BD013C65426C41A0256442ED01BA
:101AE0002C40084D1B186419074D0633013A92B279
:101AF000AA42EDD01888461C1E80085C2070F5E7CD
:101B0000B067FF1F00400040FFFF00000F220E4B98
:101B100010B59868104002380A280BD801F0FEFF73
:101B20000D0A0B0A0A110A0A0A0A060002210020FD
:101B3000FFF762FF10BD0121F9E70020FFF794FFD6
:101B4000F8E7DB6FF6E7C046004000400F220E4B7F
:101B500010B59868104002380A280BD801F0DEFF53
:101B60000E0A0B0A0A120A0A0A0A060002210120BA
:101B7000FFF742FF10BD01210800F9E70120FFF740
:101B800073FFF7E7DB6FF5E70090004013B5334CC8
:101B90002378072B3DD8324B1A78324B002A39D1A3
:101BA0008022196852020A431A60252001F0C0FE03
:101BB00020232D4A11680B43802113606B460422B9
:101BC000C90508680733104228D080210422C905BE
:101BD000C86810422ED080212020C905CA688243DF
:101BE000CA6014221A701A78002A2FD18021C905E0
:101BF000C86820320243CA6014221A701A78002A78
:101C000028D11A4B1A7D22785A601D221A70593237
:101C1000DA6013BD1A6816490A40C5E7086802432E
:101C20000A6014221A701A78002ACED01A78013A63
:101C3000D2B2F7E7C8680243CA6014221A70197852
:101C40004A1ED2B21A700029F9D1C4E71A78013AB3
:101C5000D2B2C7E71A78013AD2B2CEE75043FF1F9B
:101C60001844FF1F3CF000404843FF1F0020004085
:101C7000FFFFFEFF564B70B51B68012B03D1554A81
:101C8000936D0133936502F08FF9534B534A1860FB
:101C9000534B544C1A600123534A1360534A136048
:101CA0002378002B06D006225149524801F074FFD8
:101CB00000232370504A514B10681B78C1B2002B8F
:101CC0000ED14F4CC0B223785BB2002B4FDB237890
:101CD00024785BB264B21B0424021B191B18136026
:101CE0000B1C50294ED95023464A47491078DBB285
:101CF000FF2202284BD10868444C454D267890437A
:101D00002A78964254D9227824782E78023B5D10A6
:101D1000A31B6B435201D31A10335B1118430860A5
:101D200001F072FF031F012B45D83A4B1B78002BA3
:101D300006D0394B1B78002B02D0002002F01CF992
:101D4000A122364B92009978354B4A431B689B1869
:101D5000832292009B181B78033B012B03D8AF20F2
:101D6000400002F041F901222E4BDA8270BD237847
:101D700024785BB264B2FF33FF341B0424021B19C6
:101D80000138ABE7CAB2022AAED20223ACE7086838
:101D9000254C264D267890432A78964208D92278F9
:101DA00024782D78023B5B10641B63435201B2E739
:101DB0002378DBB2B2E70228D5D11D4B1B78013B5B
:101DC000022B03D91B4B1B78022BCCD16C20C8E70C
:101DD0009809FF1FFC0FFF1F3C64FF1FFF3F00001F
:101DE000141003404064FF1F0C1003400010034018
:101DF000D50BFF1F7211FF1FB40003408C09FF1F9A
:101E0000680AFF1F490AFF1F94000340460AFF1F8C
:101E1000470AFF1FF908FF1F2209FF1F300DFF1F90
:101E20003409FF1FBC0BFF1F440AFF1F450AFF1F99
:101E30001C09FF1F2309FF1F10B502F035F800220F
:101E4000014B1A8010BDC0463A64FF1F10B502F066
:101E500043F8A121054A89009478054A6143126834
:101E6000044B5218528C1A8010BDC046300DFF1F13
:101E70003409FF1F3A64FF1F10B50D4B0D4A9978C6
:101E8000A1239B004B431268D218531DD97F0A4BE4
:101E90001B88994209D2441C07D0C82805D0D269B2
:101EA0005B1A5A43054B5343C01801F00DFF10BD98
:101EB000300DFF1F3409FF1F3A64FF1F710200003D
:101EC00070B5244D2B68002B28D001F035FF2B680E
:101ED000D8402B680400002B27D001F055FE2B685A
:101EE000D8401D4B1D4A9978A1239B004B43126893
:101EF000D118D25C91239B00002A20D0CA5801320D
:101F0000CA50174B17491B680868834214D3D23B49
:101F1000181A012A1AD0144B186070BD01F00CFF7A
:101F2000124B196801F028FED3E701F02DFE0F4B8C
:101F3000196801F021FED4E70D495B18E8E7CA50A3
:101F40000C4B1B68DB68E418201AE4E7F530FF301F
:101F5000E1E7C0461C08FF1F300DFF1F3409FF1FBB
:101F60009C09FF1F3C64FF1FA009FF1F1808FF1FEB
:101F70002DFF3F004464FF1F70B504000D002829A9
:101F800016D10300A433C2881B889B1A0B4A9BB24C
:101F900093420DD906006A3605223100653001F002
:101FA00053FF002804D13100200001F04DFE70BD28
:101FB0002900200001F0C8FEF9E7C046FE7F0000BE
:101FC000F8B50500012001F097FF134CA36AA26A3F
:101FD0009342FBD1114E336001F08EFE1049030095
:101FE00008601048426894460F4A17680022BC45B2
:101FF00001D24268BA1A0D4802603268AD18A422B4
:10200000E562606A520302436262094A1278002A5A
:1020100001D00F3B0B60F8BD00F00040340AFF1FF9
:10202000E408FF1F28100040180AFF1F1C0AFF1FAA
:102030001C09FF1F70B580241025E405A3682B43FD
:10204000A36001F0C9FEA368AB43A36070BD0000AC
:10205000F7B5160080221C001023D205019191686B
:1020600005000B43936000225A4BD7301A6001F0F1
:102070007BFD9D232A002F009B00EB58CA320121D3
:102080000092FC37002B01D00021009A386801F043
:10209000E3FD2900009BCB311A784F4BD3351A60F2
:1020A0004B780A781B0213438A7812041A43CB78C0
:1020B0001B061343494A1BBA13604B790A791B026A
:1020C00013438A7912041A43CB7931001B06134358
:1020D000434A1BBA13606B782A781B021343AA7811
:1020E00012041A43EB781B0613433E4A1BBA1360D3
:1020F000019A330213433C4A13603C4B22001B1BE2
:102100009C4603293DDCB3089A0013005142B21AE1
:10211000032A46D1354AE018511A827840781204D1
:1021200000020243E05C043302430A600022FF2BFA
:102130004BDDF0222E4B12011A600F222D4B1A603C
:102140002D4A1368002BFCD00023224A2749136034
:10215000091B321D0B191B68043A180A23706070A2
:10216000180C1B0EA070E3700434002AF2DC8022ED
:1021700010213B68D20501333B6093688B43936029
:10218000F7BD6346D578981893782D061B042B432A
:10219000157804392B43557804322D022B43036004
:1021A000AFE7022A0AD1114AE05C511AE2185278CC
:1021B000120202430A6004339BB2B7E7012AB5D189
:1021C0000A4A521AE15C1160F5E7084959180A6099
:1021D0000433ACE7000004403C00044038000440F5
:1021E00034000440300004400C000440000104406E
:1021F000040004401000044014000440F7B515002A
:1022000080221C001023D2050091916807000B4327
:1022100093600023654AD730136001F0A5FC9D232D
:102220003E009B00F9583B00CA363200FC330029BF
:1022300000D07FE0586801F00FFD390032785C4B28
:10224000CB311A604B780A781B0213438A78AC466C
:1022500012041A43CB78281D1B061343554A1BBA98
:1022600013604B790A791B0213438A7912041A43CB
:10227000CB791B061343504A1BBA13604B7A0A7A78
:102280001B0213438A7A12041A43CB7A21001B06DD
:1022900013434A4A1BBA1360009A2B021343484A5D
:1022A00013602200474B1B1B0093009BCE785B18EA
:1022B00001938B7836061B0433430E78043833437E
:1022C0004E78043136023343019E33600328ECDC40
:1022D0000321A808431C9B002940800003292BD11F
:1022E0003849E5185E18A9786D78E35C09042D0279
:1022F000294319433160030008330021FF2B2DDDF2
:10230000314B324919600F21314B196001232749A4
:102310000B60304B19680029FCD006211B680B406C
:10232000042B20D080220020D20593680A318B43F1
:102330009360FEBD01217DE7022908D121495D1886
:10234000E1184978E35C090219432960D3E70129C0
:10235000D3D11C495918E35C0B60CCE71948181815
:1023600001600433CAE7002310490B606346002B69
:102370000CDC3B00FC335A68102101325A60802289
:10238000D205936801208B439360D2E7009B9B1892
:102390001B68190A13705170190C1B0ED37004239B
:1023A0005B4291709C440432E0E7C0460000044068
:1023B0003C00044038000440340004403000044035
:1023C0000C0004400001044004000440080F000019
:1023D000100004401400044070B5061E19D00222FB
:1023E0005A4B9B799343012B13D1594B1A78FF2AEF
:1023F0000FD15A78FF2A0CD19A78FF2A09D1DA78BE
:10240000FF2A06D11A79FF2A03D15B79FF2B00D16D
:1024100099E0504B0C201A78012A08D000224E4D2A
:102420001A7029780B00093B042B01D8212070BDBC
:102430004B1F012BFAD9454CA37B042B00D982E01A
:10244000A279032A00D97EE09A1ED2B2012A02D8CC
:1024500060881F2877D9002E56D0012E73D1A0880E
:102460000128E3D0002907D1581E032803D801F022
:1024700055FB121715122E702978481E032811D803
:102480000025364B1D602823237501F0B5FBA842BB
:1024900027D0A580CAE702212970EDE70421FBE7D8
:1024A0000321F9E707390129C0D82D490968C96A0C
:1024B0008906BBD52B4908780028B7D1012A01D954
:1024C000002BB3D102230B708021274D26338901C5
:1024D0002878237501F018FC80212878890101F003
:1024E0001BFC0123A380214B1B78002B0AD0FA226E
:1024F00080211F4B92001B8809025A431A4B1878FF
:1025000001F08AFD002092E701F08EFD2B78A68075
:10251000073B012B03D917482E7001F0C5FB114B67
:10252000114C1A78002A06D08021002220788901D7
:102530001A7001F0E9FB01F097FB80212078090275
:1025400001F0E2FBDEE7122071E7C046A60BFF1F99
:102550006B09FF1F1A09FF1F1C09FF1F4809FF1FF6
:102560004464FF1F2309FF1F1B09FF1F2109FF1FD1
:102570002C09FF1F0010004010B5002901D001F008
:102580007BFB10BDF7B5604B01919978A1239B00AF
:102590004B435E4A060014681022E418D6235B0001
:1025A000E0583623FF33E35C00279343222B41D1CD
:1025B000574B0F3A1A600760012501F005FC019B9B
:1025C0001880E8235B00E35C002B01D0B34258DDA8
:1025D0000023504FFB70AD33FF33E3581A68002AD5
:1025E00003D09B88DB439B071DD03823FF33E35C7C
:1025F000002B18D09B235B00E35C002B13D1D1335D
:10260000FF33E35CB3420EDAA4235B00E15AE01827
:10261000090A023101F090FC23000122FE33013E41
:1026200001351A87FA70E8235B00E35C002B2AD09F
:10263000A8B2FEBD03683D00002BBED081880430E7
:10264000090A023101F078FCD6235B00E3581F60D1
:10265000B2E72300B133BA00FF33985801378188BD
:102660000430090A023101F067FCE8235B00E35CF7
:10267000BB42EEDCE822F61AED1800235200A35408
:10268000A6E70027F1E7200001F04EFB00281FD04D
:10269000002E1DDD7319882647190193B60020000E
:1026A00001F01AFB5A3080002018406801358188FB
:1026B0000430090A023101F03FFC200001F04CFB1C
:1026C000A3590133A351BD4202D0019B9D42E6D1E3
:1026D000114BE35C002BABD095239B00E35C002BFC
:1026E000A6D00E4BE15A0029A2D00D4AA35C994214
:1026F00002D90133A3549BE700231A212000A354DD
:1027000001F05AFB94E7C046300DFF1F3409FF1F4C
:1027100000140340E010FF1F5A0200007202000084
:102720005E0200000D4970B54A6E0D4CD2038B69F4
:10273000D20BA24206D80B4D0224AA4204D901F0C2
:1027400043FC70BD02246442E21815007E2425403B
:102750002242F4D0A3432B438B61F0E700F000400A
:102760000A200000FC1C0000F8B51D4B1D4F1A7814
:10277000002A10D1BA7B002A02D101321A7003E07C
:10278000032AFAD0022AF8D001F036FA00220120FA
:10279000154B1A70F8BD154B154D1C68154B9E78DE
:1027A00001232B702878C0B200F09EFBBB7B002B6E
:1027B0000BD101F019FAA1239B007343E418832382
:1027C0009B00E41823782B70E4E7032B02D101F07F
:1027D0001BFBF0E70020022BDCD101F0B5F9EAE7A2
:1027E0001C09FF1FA60BFF1F2309FF1F3409FF1F32
:1027F000490AFF1F300DFF1FF0B587B00EAD2F78CF
:102800000FAD2D780593AC46634614000E4D0CAA0F
:1028100012782E7803930D9B009201932200059B62
:10282000029701F0E9FA2E70012C01D0042C08D196
:10283000802206498B889343054A1278D2011343BC
:102840008B8007B0F0BDC0461C09FF1F6C11FF1F35
:102850007809FF1F0B001B3B70B504003020E02BF4
:102860000DD81300E025493BFF3B9BB2ED00AB4286
:1028700005D8034B200019825A8201F085FA70BDF9
:102880008410FF1F10B501F08FFB054B00205B6823
:10289000052B04D9034A5268D20200D4980810BD0F
:1028A00000100040FCE100E070B501F0BDFB0D4BF5
:1028B0001B68FC33DC691D6AFFF7E4FF641984427E
:1028C00004D2094B01241B68002B07D004220024EA
:1028D000064B1A70064A93690133936101F0C4F9FB
:1028E000200070BD4464FF1F9809FF1F2309FF1FCC
:1028F000FC0FFF1F70B50C4D2B68FC335C6A01F0B8
:1029000093FBFFF7BFFF2B680025FC339B6AE3189E
:10291000834204D2054B1B68AB4200D1051B01F07A
:10292000A3F9280070BDC0464464FF1F9809FF1F2B
:10293000D722044B92009B5810B5002B00D098472B
:1029400010BDC0460000FF1F10B501F0CFF8FFF723
:10295000EFFF2749274BCA6D274C1A4084235B00A1
:102960001343CB65254B1B68186A01F0C5FA244B4D
:10297000244A1A60244B254A1A60A022244B520094
:102980001A60244B187801F0BFFA2000224901F0A8
:1029900003FA0023A3600233A360204B2049236085
:1029A00003232048A36001F0F7F910221E4BFF20FB
:1029B0001A60802252031A60802292031A608022D9
:1029C00012041A6001F0D8FA012001F08DF9FA2002
:1029D000400001F049FA582001F006FB134801F0CD
:1029E0001BF9012001F0E8F8072001F09DFA10BD65
:1029F00000F0004000FEFEFF141000404464FF1F82
:102A0000000003400180063DBC0003403408000084
:102A1000A40003404A0AFF1F71020000C30900001E
:102A2000FFFF3F002810004000E100E0307500008B
:102A3000674E336888331B6883F3088801F01CFAFB
:102A4000644A6549136800200B401360634B644A75
:102A50001B68934200D1A6E001F0BEF80221614A52
:102A600013688B431360FFF76FFF5F4B5F4C187861
:102A7000C0B201F0C1FA0023A3600233A3605C4B33
:102A80000120236001F038FA0323A36001F014FA57
:102A9000040001F089FA050001F00EFA554B1860A8
:102AA00001F0BAF9544B1968621A531EA14200D2C0
:102AB00013008022D203934201D39B029B0A326807
:102AC000D16AC90700D471E04C491C0C09689BB25B
:102AD0004C4359432402090A641803264849FC322E
:102AE00093680A6847489B1A474A0768126847492B
:102AF0009B18474A9A1833409208DB190A60036012
:102B0000042B03D9013233400A6003600E68414947
:102B1000A619300001F030F83F4F3E493B68C3181A
:102B20003B603000019301F097F93C4E3068081883
:102B300038493060884205D9019B01333B6001F080
:102B40008BF9316001F078FA354B1B78002B0DD0F2
:102B500001F02AFA334B621B196812188A4232D2EA
:102B60004919091B091A304801F016F92F4E337A1A
:102B7000002B0ED001F018FA621BF1681218914276
:102B800024D94919091B091A294801F005F900231C
:102B90003372284B83F3088801F0EEF8002001F02F
:102BA0001BF801F011F801F017F85CE7DC0199005F
:102BB0000234641A5900641A09214B438033CB4014
:102BC000A408E41889E7FA218900CCE71A49DBE771
:102BD0004464FF1F1CF00040FFFFC1FF0C0AFF1FF1
:102BE000B641210310000040490AFF1F14100040A5
:102BF000C3090000100AFF1F340AFF1F380AFF1F15
:102C0000200AFF1F280AFF1F1C0AFF1F240AFF1F9C
:102C1000C4090000710200006008FF1F2C0AFF1F9A
:102C20001C09FF1FE408FF1F00100040740BFF1F6A
:102C30003C10004000000020DC050000A022054BF5
:102C400092009B5810B5002B01D0984710BD01F0A1
:102C5000C3F9FBE70000FF1FA122054B92009B5820
:102C600010B5002B01D0984710BD01F0B5F9FBE776
:102C70000000FF1FA222054B92009B5810B5002BAD
:102C800001D0984710BD01F0A7F9FBE70000FF1F36
:102C9000A322054B92009B5810B5002B01D09847FA
:102CA00010BD01F099F9FBE70000FF1FA422054BBE
:102CB00092009B5810B5002B01D0984710BD01F031
:102CC0008BF9FBE70000FF1F70B501F06DF94F4B6A
:102CD000186001F069F80400C30702D401F0DCF8C1
:102CE00070BD00224A4B1A604A4B187801380428FC
:102CF00029D800F013FF0320181C2400200000F046
:102D000053FF0128ECD0444C2378042B6ED101F002
:102D1000EBF80028E4D001F03FF9582001F064F905
:102D200002232370DCE7200001F046F9E9E72000E8
:102D300001F01AF8E5E7200001F026F9E1E72000AC
:102D400001F0C2F8DDE700F05FFF0500012808D1BF
:102D5000324B1B78053B012B03D82000FFF76EFF99
:102D6000D1E72D4B1B78022B01D0052B20D1022D52
:102D700028D12B4B9B7BAB431CD12000FFF76CFF72
:102D8000264B18780128BED16405BCD424492522DD
:102D90004B7B034205D1233A13405A425341263319
:102DA0001A000B7D9342AED9322001F0D5F8AAE784
:102DB000022D07D1194B1B78052B11D12000FFF7ED
:102DC00059FFDDE7012D0BD1012B03D12000FFF7C7
:102DD0005FFF98E7062B03D12000FFF767FF92E71C
:102DE000200001F0F9F8022D8DD1C9E7032B04D1A1
:102DF0000C4B987C00F0F8FF72E7072B00D06FE7D0
:102E0000094B987B00F040FF6AE7C0469C09FF1F12
:102E10009809FF1F9009FF1F2309FF1F1C09FF1FAF
:102E2000A60BFF1FBC0BFF1FD40BFF1FFA210A4B81
:102E30000A4A49001A640A4A5A500A4A04395A503E
:102E4000094A08319A64094A5A50094A5C315A5071
:102E5000084ADA667047C0460000FF1FF927FF1FC7
:102E6000F528FF1FA928FF1FD923FF1F6927FF1F70
:102E7000791EFF1F4D1EFF1FF7B50B0CFF27012208
:102E8000009300233C001E001D009446019089B26F
:102E900062469A401000084018413618B6B2FF2F1B
:102EA00002D1012E00D19FB2009802401A41AD1804
:102EB000ADB2FF2C02D1012D00D19CB20133102BF9
:102EC000E6D10320012E07D1012D04D1019B24015D
:102ED000E4191C700138FEBD102EFCD10238102DF3
:102EE000F9D00230F7E700008023F7B59C46264B67
:102EF000264F01932649274A274D284C284B022864
:102F00001AD1604638600868264E30408026360365
:102F10003043086001990978002909D11660224AD6
:102F20002A60224A2260E02219689143A03A1BE0FD
:102F30008021C9021160F2E766463E600F68194EB3
:102F40003E408027FF023E430E6001990978002928
:102F50000DD1176001280ED1154A2A60154A22604A
:102F6000E02219689143C03A0A431A60F7BD8021F4
:102F700089021160EEE7E0210F4A02432A600F4AFE
:102F800022601A688A43F0E74B0AFF1FE000034003
:102F9000D80003409000034000000340500003406D
:102FA00040000340FFFFE3FF0280063D804508220A
:102FB0000180063D80660822008006988055082220
:102FC000F8B51E4B80261A680020140034403242A7
:102FD00032D11A681A4F32431A6001223B68063018
:102FE00093433B6000F088FF0122164D2B681E437F
:102FF0002E603B680A2613433B608027BF00124BBC
:103000001B683B4211D1013EF6B2FF2E09D17E2250
:103010000E4B1C682B68E40B1440934323432B6036
:1030200005E0082000F068FFE9E7002EEFD18022DC
:103030002B68600893432B60F8BDC046C4F0004085
:103040005CF0004018F0004068F0004060F0004084
:1030500010B500F0E9FE01215820034A00F084FF7A
:10306000FFF7AEFF10BDC046600AFF1F10B5782203
:103070000021034800F0C8FF00F066FF002010BDEB
:103080003867FF1F70B5040000F0CEFF00230C204E
:103090000B4A010059438D18515C00290DD0A14203
:1030A00008D1012300246B7000F006FE00F0DCFD67
:1030B000200070BD01330A2BEBD11224F6E7C04685
:1030C0003867FF1F70B5040000F0AEFF0023190041
:1030D0001D000D4A1078002806D0A0420CD1557072
:1030E00001310C320A29F5D1002B0AD100F02CFF56
:1030F00000F0BAFD002070BD5078461EB0411B188C
:10310000EEE700F0D9FDF3E73867FF1FF7B50400DD
:103110000C20002384460E4D019267465F43E85D14
:103120007E19A04212D000280BD10A4B9C46624661
:103130001B7808331370019B70707C557160B3600D
:10314000FEBD01330A2BE8D10320F9E70720F7E79A
:103150003867FF1F3467FF1F8020F8B5484BC00554
:103160001B68C1248360474BFF251A680123134362
:103170004361454BA4001A68444B40211A60444BFC
:103180001A68444B1A60444B1A59AA431A51C52273
:1031900092009E58AE433143802699509F583F4934
:1031A000F6010F403E439E509E5880273602360A55
:1031B0003043985080201A5900020A4002431A51A5
:1031C00004341A59364E3F04324080263A431A518D
:1031D0001A5936061202120A32431A5108341A5981
:1031E00080260A4002431A51C32292009F58B446D7
:1031F000AF4337439F509F58294E0F4007439F507E
:103200009F58374080263604374380269F509F586A
:1032100036063F023F0A37439F50C0221F59AF4333
:103220003A431A511A591202120A1643C6221E5163
:1032300092009C58AC4365462C439C509C580025FA
:103240000C4020439850C72080001A58154C11405C
:10325000C02212020A431A50134B1B78DB08AB4200
:1032600001DC0020F8BD2378002B06D0A368002BDA
:1032700000D0984701350C34EEE71220F2E7C04643
:103280004C43FF1F4843FF1FB0F000403067FF1F53
:10329000B4F000402C67FF1F00E100E0FF00FFFFDB
:1032A000FFFF00FF3867FF1F3467FF1F030010B5E3
:1032B0001F2809D8072200201340072404490A7850
:1032C000A24313430B7010BD00230620F5E7C04650
:1032D0003467FF1F054B06491B780A6805485B07E2
:1032E00002401B0B134300200B6070473467FF1F25
:1032F0001CF00040FFFFC1FF70B50C25FFF7EAFF8F
:103300000A4B1C780A4BE4086543ED18002C01D1E8
:10331000200070BD2B78002B06D06B68002B00D0EE
:103320009847013C0C3DF1E71220F2E73467FF1F9C
:103330002C67FF1F1FB5002102220B000191009195
:10334000052000F0A9FC02230B490A681A42FCD1AF
:1033500020230393039B5A1E0392002BFAD1074AA2
:103360001368002BFCDA0B246C442000012100F0D0
:1033700063FC207804B010BD90C8004000C8004035
:1033800013B504000A4B0193019B002B01D11120BE
:1033900016BDFFF7CFFF23000340044205D00520F0
:1033A00000F0AAFD019B013BEDE71800F0E7C046E5
:1033B000FFFFFF0707B500F037FE80220821D20586
:1033C000936A0191002B01D10739916202210C4AC5
:1033D00011600199481E01900029FAD10331116052
:1033E000053101910199481E01900029FAD111601F
:1033F000002B02D18022D205936200F035FC07BD7C
:1034000000C00040F0B52D4C89B02378002B4FD17F
:10341000FEF7D2FA02232A4F03903A681A42FCD1EF
:1034200020230693069B5A1E0692002BFAD1254EA6
:103430003368002BFCDA0120FFF7A2FF011E02D047
:10344000112009B0F0BD030003220190009005ADEA
:103450009F2000F021FC0321280000F0EDFB022357
:103460003A681A42FCD120230793079B5A1E079201
:10347000002BFAD13368002BFCDA0120FFF780FF24
:103480000028DDD10398FEF7ABFAAA786B78110417
:103490001B020B4329780B4363601300113B0A495D
:1034A000052B07D801239340A3600B6001232370F1
:1034B0000020C6E780231B03F6E7C0463443FF1F06
:1034C00090C8004000C800409808FF1F1E4B30B550
:1034D0005A6818781D4B85B0D31859424B410121C9
:1034E0000093002300F0A0FB194B1A4A02259A63AF
:1034F00000221A6510325A658022C4219D65164B40
:103500001648D202DA6789004258154B80241A40C7
:1035100080231B0413434350642341200393E40599
:1035200000F006FA402000F003FA6562039D6B1E6E
:103530000393002DFAD103236362FFF73BFFA562DB
:10354000FFF760FF05B030BD4043FF1F95FFFEF75A
:1035500000C80040050001FF04E100E000E100E0D8
:10356000FFFF00FFF0B585B00700FEF725FA022344
:1035700005002D4C22681A42FCD120230093009BA9
:103580005A1E0092002BFAD1284E3368002BFCDA29
:103590000120FFF7F5FE002803D01124200005B01C
:1035A000F0BD234B2360022322681A42FCD1202362
:1035B0000193019B5A1E0192002BFAD13368002B14
:1035C000FCDA0120FFF7DCFE0028E6D1194B1F6072
:1035D000022322681A42FCD120230293029B5A1E26
:1035E0000292002BFAD13368002BFCDA0120FFF79E
:1035F000C7FE0028D1D1104B2360022322681A4253
:10360000FCD120230393039B5A1E0392002BFAD173
:103610003368002BFCDA0120FFF7B2FE041EBCD198
:103620002800FEF7DDF9B9E790C8004000C8004067
:1036300001000006A8C800400180000110B500206C
:10364000FFF790FF10BD000010B5064B18705960D1
:10365000FFF73CFF00211320034AFFF757FD00202E
:1036600010BDC0464043FF1FCD34FF1FF0B504001E
:1036700085B003920291FEF79FF9882263035B0BEA
:1036800052051A438023DB059D6A8023274F009251
:10369000BA68002601901B039A420CD9F823260031
:1036A0001B041E401C4206D08022214B52025E6247
:1036B00019680A431A60002D0BD100F0B5FC0222F4
:1036C0001C4B1A608023DB055A62013A9A6200F0B3
:1036D000CBFA0023039A934220D1002D0AD100F0A7
:1036E000A3FC144B03221D608023DB055A629D62FC
:1036F00000F0BAFA8023BA681B039A4208D9002E58
:1037000006D000220A4B0C495A621A680A401A6015
:103710000198FEF765F9002005B0F0BD009A029906
:10372000D2181278CA540133D4E7C0463443FF1F7D
:1037300000C8004000C00040FFFFFEFFF0B587B0AA
:10374000029103920400FEF737F9019000F06CFC3F
:10375000802302250122234EDB0535605D629A62DB
:1037600000F082FA204F3B682B42FCD120230493C7
:10377000049B5A1E0492002BFAD11C4D2B68002B7F
:10378000FCDA0120FFF7FCFD002802D0112007B071
:10379000F0BD2000039A029900F0BEFB0223040052
:1037A0003A681A42FCD120230593059B5A1E0592C4
:1037B000002BFAD12B68002BFCDA0120FFF7E0FD8B
:1037C000051EE3D100F030FC80230322DB053560C9
:1037D0005A629D6200F048FA0198FEF701F9E0B2E2
:1037E000D5E7C04600C0004090C8004000C8004077
:1037F000F0B5802489B00600FEF7DEF8E405A36A80
:1038000002250393029000F00FFC0123304F3D602E
:103810006562A36200F028FA2E4C23682B42FCD18B
:1038200020230593059B5A1E0592002BFAD12A4DA1
:103830002B68002BFCDA0120FFF7A2FD002803D043
:103840001124200009B0F0BD244B2360022322681C
:103850001A42FCD120230693069B5A1E0692002B87
:10386000FAD12B68002BFCDA0120FFF789FD021E3C
:10387000E6D11B4B03211E60030001900090202025
:1038800000F00AFA022322681A42FCD1202307938F
:10389000079B5A1E0792002BFAD12B68002BFCDAEB
:1038A0000320FFF76DFD041ECAD100F0BDFB80238D
:1038B0000322DB053C605A629C6200F0D5F9039B51
:1038C000002B01D1FFF776FD0298FEF789F8B8E7E3
:1038D00000C0004090C8004000C800400100000641
:1038E00094C8004007B5000201910422000A01A912
:1038F000FFF724FF0EBD000073B5050005240B4A39
:10390000A3005B429B1819686B46DE1D3000FFF771
:10391000B3FA022804D133782B55013CEFD276BD9F
:10392000052CFCD00128FAD10230F8E71409001167
:103930001F2807D8012380228340D20591680B43BA
:10394000936070473F2808D80123802220388340A5
:10395000D20551690B435361F3E75F28F1D8012386
:10396000802240388340D205116A0B431362E8E796
:103970001F2807D8012280218240C9058B68934304
:103980008B6070473F2808D8012280212038824070
:10399000C9054B6993434B61F3E75F28F1D80122D6
:1039A000802140388240C9050B6A93430B62E8E7E7
:1039B0001F2810D880230200DB05153A1968012A58
:1039C00006D820229143196019680A431A6070478B
:1039D00001228240F6E73F2811D880230200DB0550
:1039E000353AD968032A06D810229143D960D9689C
:1039F0000A43DA60EBE7012220388240F5E75F28CE
:103A0000E5D842238022181A413B8340D205516AEF
:103A100099435162516A0B435362D8E710B50400D1
:103A2000012813D1A022184992050B685B015B099C
:103A300013430B60154B164A19681140154A0A4387
:103A40001A60402219680A431A6010BD0028FCD190
:103A500001000A2000F018FA21000B2000F014FAEF
:103A6000C0220A4B920019680A4340211A601A6862
:103A70008A431A60B022044912060B685B015B0995
:103A800013430B60E1E7C04614F000401CF0004017
:103A90007F00FEFF80FD010072B6074A1368013304
:103AA00013600422054B1A600023054A136080222C
:103AB000D2055360FEE7C0467808FF1FC0F0004003
:103AC000C4F0004005490B68002B05D1044A0A6088
:103AD00004490A60044A13607047C046140AFF1F75
:103AE000841E0000380AFF1FC4F000400023034A70
:103AF0001360034A1360034A1360704754F0004098
:103B000040F1004044F1004002B4714649084900C8
:103B1000095649008E4402BC7047C04602B4714643
:103B200049084900095C49008E4402BC7047C04600
:103B300003B47146490840004900095A49008E44BF
:103B400003BC70470000000001B40248844601BC79
:103B5000604700BF19FA000001B40248844601BC66
:103B6000604700BFE927000001B40248844601BC59
:103B7000604700BF8944000001B40248844601BC8C
:103B8000604700BF090E000001B40248844601BC32
:103B9000604700BF6D0B010001B40248844601BCC0
:103BA000604700BFE94C010001B40248844601BCF3
:103BB000604700BF0134010001B40248844601BCE3
:103BC000604700BFE512010001B40248844601BC11
:103BD000604700BF8552010001B40248844601BC21
:103BE000604700BF016C010001B40248844601BC7B
:103BF000604700BFE9F6000001B40248844601BCFA
:103C0000604700BFA9D8000001B40248844601BC47
:103C1000604700BFDD0C010001B40248844601BCCE
:103C2000604700BF8D11010001B40248844601BC09
:103C3000604700BFC56D010001B40248844601BC65
:103C4000604700BF3D71010001B40248844601BCD9
:103C5000604700BF85C1000001B40248844601BC32
:103C6000604700BF2144000001B40248844601BC03
:103C7000604700BF9DA9000001B40248844601BC12
:103C8000604700BFE9D4000001B40248844601BC8B
:103C9000604700BFC1F7000001B40248844601BC80
:103CA000604700BF496D010001B40248844601BC71
:103CB000604700BFC1A5000001B40248844601BCB2
:103CC000604700BF21A9000001B40248844601BC3E
:103CD000604700BF8937010001B40248844601BC37
:103CE000604700BFD9B0000001B40248844601BC5F
:103CF000604700BF6911010001B40248844601BC5D
:103D0000604700BFBD5C010001B40248844601BCAD
:103D1000604700BFB352010001B40248844601BCB1
:103D2000604700BF0D52010001B40248844601BC47
:103D3000604700BF71B0000001B40248844601BC76
:103D4000604700BFE90B010001B40248844601BC92
:103D5000604700BF51B8000001B40248844601BC6E
:103D6000604700BF5976010001B40248844601BC97
:103D7000604700BF0534010001B40248844601BC1D
:103D8000604700BF7997000001B40248844601BC37
:103D9000604700BF116E000001B40248844601BCB8
:103DA000604700BF2D6C010001B40248844601BC8D
:103DB000604700BFBD0B010001B40248844601BC4E
:103DC000604700BF53B9000001B40248844601BCFB
:103DD000604700BFCD0C010001B40248844601BC1D
:103DE000604700BFDD3F000001B40248844601BCCB
:103DF000604700BF4DF9000001B40248844601BC91
:103E0000604700BF9D6A000001B40248844601BCBF
:103E1000604700BF75F8000001B40248844601BC49
:103E2000604700BFC166010001B40248844601BC7E
:103E3000604700BFED68010001B40248844601BC40
:103E4000604700BFF5B5001101B40248844601BCCB
:103E5000604700BFCD4C010001B40248844601BC5C
:103E6000604700BF090E000001B40248844601BC4F
:103E7000604700BF8512010001B40248844601BCBE
:103E8000604700BFC9A9000001B40248844601BCD4
:103E9000604700BF4DA2001101B40248844601BC36
:103EA000604700BFDD0A010001B40248844601BC3E
:103EB000604700BF8D82000001B40248844601BC07
:103EC000604700BF156B010001B40248844601BC85
:103ED000604700BFF935010001B40248844601BCC7
:103EE000604700BFF9ED000001B40248844601BC00
:103EF000604700BF01D7000001B40248844601BCFE
:103F0000604700BF0189000001B40248844601BC3B
:103F1000604700BFEDA5000001B40248844601BC23
:103F2000604700BF9573010001B40248844601BC9C
:103F3000604700BFF90D010001B40248844601BC8E
:103F4000604700BFC115010001B40248844601BCAE
:103F5000604700BFADAE000001B40248844601BC1A
:103F6000604700BF6137010001B40248844601BCCC
:103F7000604700BF0167010001B40248844601BCEC
:103F8000604700BFED6B010001B40248844601BCEC
:103F9000604700BFF535010001B40248844601BC0A
:103FA000604700BF6DF6000001B40248844601BCC2
:103FB000604700BFC95C010001B40248844601BCEF
:103FC000604700BF0934010001B40248844601BCC7
:103FD000604700BFD1AE000001B40248844601BC76
:103FE000604700BFE917010001B40248844601BCE4
:103FF000604700BF7912010001B40248844601BC49
:10400000604700BF8914010001B40248844601BC26
:10401000604700BFB70E000001B40248844601BCEF
:10402000604700BF8B52010001B40248844601BCC6
:10403000604700BF75A9000001B40248844601BC76
:08404000604700BFD5440100F8
:10404800020000009ABE001101000000A8BC001187
:104058000200000096BE0011010000008840FF1F0A
:1040680002000000B0BC001101000000C861FF1F81
:104078000200000094BE0011030000003C61FF1F15
:1040880012000000020000009ABE001101000000AA
:10409800F0BC00110200000096BE001101000000F3
:1040A800EDBC001102000000FABC00110300000082
:1040B8007761FF1F0200000094BE0011030000009A
:1040C8008C61FF1F0200000096BE00110100000075
:1040D800ECBC001102000000F8BC00110300000055
:1040E8004D61FF1F0200000094BE00110300000094
:1040F8006E61FF1F020000009ABE0011010000005F
:1041080034BD00110200000096BE0011010000003D
:10411800D141FF1F0200000046BD00110100000050
:104128002BBD00110200000096BE00110100000026
:10413800D041FF1F0200000044BD00110100000033
:104148009461FF1F0200000096BE001101000000EC
:10415800CF41FF1F0200000042BD00110100000016
:104168001BBD00110200000096BE001101000000F6
:10417800CE41FF1F0200000040BD001101000000F9
:1041880016BD00110200000096BE001101000000DB
:10419800CD41FF1F020000003EBD001101000000DC
:1041A80011BD00110200000096BE001101000000C0
:1041B800CC41FF1F020000003CBD001101000000BF
:1041C8000CBD001102020202020200000000000001
:1041D80016150000A54B00116B4B001188BD00118E
:1041E80090011D0018001800FFFF070102030405D5
:1041F80006020106000000000000000000000000A8
:1042080000000000000000000000000000000000A6
:1042180003000000020000009ABE00110100000027
:10422800A8BD00110200000096BE001101000000A8
:104238008C42FF1F02000000B2BD00110100000007
:10424800C261FF1F0200000094BE001103000000BD
:104258002C64FF1F0200000096BE00110100000040
:104268008C42FF1F02000000B0BD001101000000D9
:10427800C461FF1F0200000094BE0011030000008B
:104288002464FF1F120800000000000000C6C600DA
:1042980000000000000000001311000000010000F1
:1042A80000000111FFFF00005048593600000000CF
:1042B800000000000B000500F0000000B40000281A
:1042C800002800283075A000A000A000A000000869
:1042D8000008E001F00010001000100010001000AD
:1042E800100050005000500010001000D0070000CF
:1042F800000000000F0001000500307507001000E5
:10430800010081FF00000000FF000000357400116B
:104318003D720011CD6F0011FFFF0100FF0000008A
:10432800519E0011CD9B0011E59A0011000000007C
:104338000000000000000800040000003B00010825
:104348005902E00188212800FF0000000200000057
:104358009ABE00110100000060BF001102000000B9
:1043680096BE001101000000D143FF1F02000000AB
:1043780092BE001101000000F067FF1F020000005C
:1043880096BE001101000000D043FF1F020000008C
:1043980090BE001101000000CE43FF1F0200000084
:1043A80096BE001101000000CC43FF1F0200000070
:1043B8008EBE001101000000C443FF1F1800180042
:1043C8001D0090010200000302020000020000002C
:1043D8009ABE00110100000074BF00110200000025
:1043E80096BE0011010000001444FF1F02000000E7
:1043F8008CBE001100000000000000000200000058
:0E44080094BE0011030000001068FF1F20FF8B
:040000051FFF184180
:00000001FF
